:1000000067C5000082C5000080C500000C940A325C
:100010007CC500007AC5000078C5000076C50000E8
:1000200074C5000072C500000C94E52E0C94CD2F11
:100030000C94821C6AC5000068C5000066C50000FB
:1000400064C5000062C5000060C500005EC5000018
:100050005CC500000C94C12E58C5000056C50000B8
:1000600054C5000052C5000050C500004EC5000038
:100070004CC500004AC5000048C5000046C5000048
:1000800044C5000042C5000040C500003EC5000058
:100090003CC500003AC5000038C5000036C5000068
:1000A00034C5000032C5000030C5000005010980DC
:1000B000A101850319012AB700150126B700950192
:1000C00075108100C0050C0901A101850419012AE0
:1000D000A002150126A002950175108100C005013E
:1000E0000906A1018506050719E029E71500250184
:1000F0009508750181020507190029EF15002501F2
:1001000095F075018102050819012905950575010C
:100110009102950175039101C00660FF0961A1017B
:100120000962150026FF00952075088102096315F4
:100130000026FF00952075089102C005010906A15F
:1001400001050719E029E7150025019508750181CA
:10015000029501750881010507190029FF15002680
:10016000FF0095067508810005081901290515008D
:100170002501950575019102950175039101C0094D
:10018000025B00030100A0FA090400000103010161
:100190000009211101000122440007058103080024
:1001A00001090401000203000000092111010001FE
:1001B0002222000705820320000107050303200017
:1001C00001090402000103000000092111010001DE
:1001D000226D0007058403200001120100020000C7
:1001E000000832FC87020100010200010C035300E9
:1001F0006F0066006C00650000001A034A006F0083
:100200007300650066004100640061006D006300DA
:1002100069006B0000000403090446001E001F0073
:10022000200021002200290014001A0008001500F7
:1002300017002B0004001600070009000A000057F1
:100240001D001B00060019000500E300E200E000AD
:10025000777C2800A8004C002700260025002400F9
:1002600023002A00130012000C0018001C002F00AD
:1002700033000F000E000D000B00E50038003700C2
:10028000360010001100E700E600E400787C2C0046
:10029000447E3A003B003C003D003E003F00010030
:1002A0001E021F02200221022202010014142D004E
:1002B0005700340032000100351435022D1455006A
:1002C00000000100010001000100010001004500E3
:1002D0004400430042004100400001002702260282
:1002E0002502240223020000320234026402640068
:1002F000350001002E02341430142D022E000100AE
:1003000001000100010001000100010000000000E7
:10031000000000000000010000000000520000008A
:100320004A0001000000500051004F004D00010044
:1003300000000000000000000000010001000100BA
:1003400001000100010001002202610060005F0065
:100350000000010055005E005D005C0000005700D9
:1003600024025B005A0059000000560027023700A3
:1003700036006200000001000100010001000100E0
:10038000010001000000000000000000000001006A
:100390000000000000000000427801004578477826
:1003A00049784B7843780100467848784A784C7809
:1003B0000000010001000100010001000100000037
:1003C000000000000000000000000000000000002D
:1003D000000000000000007C0000500900005009EF
:1003E000000000000000AB00AE00AC000000010007
:1003F00001000100010001000100000000000000F8
:1004000000000000000000000000000000000000EC
:100410000000000000000000000000000000FC02DE
:100420000202028242428202C242424202C242426C
:100430004202020202FC0000000000000000FF0077
:100440000000000F10100F001F020200001F020228
:100450000000000000FF000000000000000001029A
:10046000020202020202020202020202020202026C
:100470000202020202010000000000000000007CF5
:100480008282824400F8242224F800FE1212120C08
:10049000004C9292926400000000000000000000F6
:1004A000000000000000000000000000000000004C
:1004B0000000000000000000000000000000FCFE42
:1004C000FEFEFE7E3E9E9E3E7EFE1E1EFEFE1E1E0C
:1004D000FEFEFEFEFEFC0000000000000000FFFF2C
:1004E000FFFFFFF0E0CFCFE0F0FFC0C0FCF9C0C0DD
:1004F000FFFFFFFFFFFF00000000000000000103FE
:1005000003030303030303030303030303030303BB
:100510000303030303010000000000000000007C4F
:100520008282824400F8242224F800FE1212120C67
:10053000004C929292640000000000000000000055
:1005400000000000000000000000000000000000AB
:1005500000000000000000000000000000000C0A85
:1005600009894929190981412111C93F0F01013127
:10057000190F8442211109050301C0A090888482CB
:1005800081909894929190F0FC838080E01CFC8094
:10059000808087F8000000000000808080808080DC
:1005A000808080808080808080808080808080804B
:1005B000808080808080808080800000000000003B
:1005C0000000FF01010101F191919161010101011F
:1005D00001FF00000000000000000000000000001B
:1005E0000000FF808080808F80818284888080806E
:1005F00080FF00000000000000000000000000007C
:100600000000FF01010101F10101010101010101EE
:1006100001FF0000000000000000000000000000DA
:100620000000FF808080808F88888888808080801C
:1006300080FF000000000000000000AE00AF0001DD
:100640000101010101010101020202020202020292
:100650000203030303030303030404040404040464
:100660000505050505060606060607070707070828
:10067000080808090909090A0A0A0B0B0B0C0C0CDB
:100680000D0D0D0E0E0E0F0F0F1010111111121275
:1006900013131414151516161717181819191A1AF2
:1006A0001B1B1C1D1D1E1E1F202021222223242453
:1006B000252626272829292A2B2C2D2D2E2F30318F
:1006C0003232333435363738393A3B3C3D3E3F40A1
:1006D0004142434445464748494A4C4D4E4F50518C
:1006E0005354555658595A5B5D5E5F616264656646
:1006F00068696B6C6D6F7072737577787A7B7D7ECD
:100700008082838587888A8C8E8F91939596989A1C
:100710009C9EA0A2A3A5A7A9ABADAFB1B3B5B7BA34
:10072000BCBEC0C2C4C6C9CBCDCFD1D4D6D8DBDD08
:10073000DFE2E4E7E9EBEEF0F3F5F8FAFDFF00DACB
:100740000281FFD9F1DB20A4A62EAF00A0C0D30008
:1007500000A1C8D30000AED580A81F408D14200092
:100760000000000000000000000000000000000089
:100770000000000000000000000000000000000079
:10078000000000007E0F00D4FFFFFFC700000078CC
:1007900000000000000000002A2B280000000000DC
:1007A0000000000000000000000000290000000020
:1007B0002C1E3420212224342627252E362D37388E
:1007C000271E1F202122232425263333362E373897
:1007D0001F0405060708090A0B0C0D0E0F10111255
:1007E000131415161718191A1B1C1D2F3130232D21
:1007F000350405060708090A0B0C0D0E0F1011121F
:10080000131415161718191A1B1C1D2F3130354CCF
:10081000814224081020408080402010082442811A
:1008200081422410080402010102040810244281BC
:1008300081C2E4F0F8FCFEFFFFFEFCF8F0E4C281A8
:100840008143270F1F3F7FFFFF7F3F1F0F274381FC
:10085000010204081020408080402010080402019A
:100860000103070F1F3F7FFFFF7F3F1F0F0703019C
:10087000804020100804020101020408102040807A
:1008800080C0E0F0F8FCFEFFFFFEFCF8F0E0C08066
:1008900000000000000000005F00000000070007EB
:1008A0000000147F147F1400242A7F2A12002313CF
:1008B0000864620036495620500000080703000013
:1008C000001C224100000041221C00002A1C7F1C49
:1008D0002A0008083E080800008070300000080860
:1008E00008080800000060600000201008040200F2
:1008F0003E5149453E0000427F400000724949494F
:1009000046002141494D33001814127F100027453D
:10091000454539003C4A4949310041211109070048
:10092000364949493600464949291E00000014004D
:10093000000000403400000000081422410014149C
:100940001414140000412214080002015909060081
:100950003E415D594E007C1211127C007F4949498D
:1009600036003E41414122007F4141413E007F49E6
:10097000494941007F09090901003E414151730085
:100980007F0808087F0000417F4100002040413F70
:1009900001007F08142241007F40404040007F0258
:1009A0001C027F007F0408107F003E4141413E0051
:1009B0007F09090906003E4151215E007F0919297E
:1009C000460026494949320003017F0103003F40A8
:1009D00040403F001F2040201F003F4038403F0064
:1009E0006314081463000304780403006159494D3B
:1009F0004300007F414141000204081020000041F3
:100A000041417F0004020102040040404040400098
:100A10000003070800002054547840007F28444415
:100A20003800384444442800384444287F0038546F
:100A30005454180000087E09020018A4A49C7800F1
:100A40007F080404780000447D4000002040403DC1
:100A500000007F102844000000417F4000007C041B
:100A6000780478007C080404780038444444380052
:100A7000FC182424180018242418FC007C08040402
:100A8000080048545454240004043F4424003C40CB
:100A900040207C001C2040201C003C4030403C009A
:100AA0004428102844004C9090907C004464544C9E
:100AB00044000008364100000000770000000041BB
:100AC000360800000201020402003C2623263C00F6
:100AD00011241FBECFEFDAE0DEBFCDBF13E0A0E0F0
:100AE000B1E0E4E9F8E602C005900D92AA38B1073A
:100AF000D9F729E0AAE8B3E001C01D92A33AB207F2
:100B0000E1F70E945D290C94E0337ACAEF92FF92DC
:100B10000F931F93CF93DF93D22F4934D8F5C42F6F
:100B2000C695C695C695477020E2C29FD001112494
:100B300070E06D59774FA60FB71F60E070E028E0B6
:100B400030E0241B3109FC01E60FF71FE4915D91B1
:100B50000E2F10E0FD0131977F01E02F042E01C020
:100B6000EE0F0A94EAF75E2BF7015083411571F0FE
:100B7000C93061F0F801022E02C0F595E7950A949C
:100B8000E2F75F965C915E2B5C935F976F5F7F4FA0
:100B90006D17C8F2CDB7DEB7E6E00C9451339C0177
:100BA00091509F31B8F4832F817034FF0BC0829530
:100BB000807F31FD806232FD806433FD8068FB01FF
:100BC0000995089531FD826032FD846033FFF7CFCF
:100BD0008860F5CF80E0F3CF982F92959F7061F4F5
:100BE00020E0982F892F8695869511F02E5F982FFB
:100BF000892F8695820F089524E0F4CF809308080A
:100C0000089580930908089521E001C0220F8A9574
:100C1000EAF780910908822BF4CF21E001C0220F6E
:100C20008A95EAF7822F8095909109088923E9CF68
:100C3000292F9A3090F5863080F590E036E0239F9A
:100C4000800D911D112451E081FD54E080FD550F70
:100C500082FD529523E0969587952A95E1F7FC0150
:100C6000EE0FFF1FE80FF91FE951F84F20E030E0C9
:100C700070E04191DF01CB01022E02C0969587956D
:100C80000A94E2F78695880B8427852384278E9320
:100C90002F5F3F4F2330310561F70895292F9A3098
:100CA00070F5863060F590E036E0239F800D911D51
:100CB0001124682F677023E0969587952A95E1F7B0
:100CC000FC01EE0FFF1FE80FF91FE951F84F40E05C
:100CD00050E080E0219130E0062E02C03695279545
:100CE0000A94E2F72170042E01C0220F0A94EAF759
:100CF000822B4F5F5F4F4330510561F7089580E0CD
:100D000008959091090821E030E0F90101C0EE0F4B
:100D10008A95EAF7D90101C0AA0F6A95EAF7EA2B8A
:100D200001C0220F4A95EAF7892F8E23E81303C0EA
:100D3000892F822B66CF2095822F8923FBCFE091CC
:100D40000F0890910E08E91302C080E008959F01FA
:100D500057E0E59FF0011124E05FF74F51815613F2
:100D600006C05081581303C05581541305C02F5F2E
:100D70003F4FF901E770E7CF81E0089580910F08B8
:100D800020910E08281301C0089501968770FACFAC
:100D900090910A088095892380930A08282F27704C
:100DA00061F4891751F090910C0892FF06C0869566
:100DB0008695869532DF10920A080895809105087D
:100DC00090910D08892B909106089115C9F0892BF7
:100DD00090918E01913021F490910B0897FD11C0F4
:100DE00096E02EE833E040E09150F90150812F5F0A
:100DF0003F4F51114F5F9111F7CF411110920608EB
:100E000008959EE126E933E0EECF8095982F8091FA
:100E100005088923809305080895803E9105D1F146
:100E2000C8F48133910509F481C048F489329105F1
:100E300009F471C08A32910509F47FC0089589339D
:100E40009105E1F082389105C9F08533910509F4E7
:100E50005DC00895843E9105D1F148F4823E91052C
:100E600031F1833E910541F181EE90E00895863E97
:100E70009105C1F1873E9105F1F1089520910B088C
:100E8000237009F064C020910C0823FF14C089E28C
:100E900090E0089520910B0820FD45C030910C088A
:100EA00030FF09C024FD24C083EE90E00895209116
:100EB0000B0822FDF7CF089520910B0822FD44C0B6
:100EC00030910C0830FD43C024FFF5CF11C02091B4
:100ED0000C0821FFF0CF80910B0884FD09C087EE3C
:100EE00090E0089520910B0823FFE5CF24FFF7CF72
:100EF00080E090E0089520910B0823FD2BC03091F5
:100F00000C0831FFE1CF84EE90E0089520910B08AA
:100F100025FFD1CFBCCF20910B0825FD1EC020910D
:100F20000C0823FFC8CF89E390E0089520910B08B7
:100F300026FFC1CF8AE290E0089520910B0826FF9A
:100F4000BACF81E390E0089582EE90E0089580EEBC
:100F500090E0089586EE90E0089585E390E008958E
:100F600090910B0892FF10C041E0282F247124308B
:100F700009F040E031E0282F2871283009F030E0F6
:100F8000431711F02CE0822793FF10C041E0282F77
:100F90002471243109F040E031E0282F28712831F4
:100FA00009F030E0431711F02CE0822730910C0853
:100FB00030FF10C051E0282F2171213009F050E09E
:100FC00041E0282F2871283009F040E0541711F033
:100FD00029E0822731FF10C041E0282F2171213103
:100FE00009F040E031E0282F2871283109F030E085
:100FF000431711F029E0822794FF02C083FD877E0A
:1010000008950F931F93CF93DF9307DFEC01D23541
:1010100008F04DC0D03508F0C3C0C03ED10530F552
:10102000CD3CD10508F09AC0C83AD10578F4C53A4C
:10103000D10508F090C0C130D10599F1CE010497D7
:10104000813A910570F1C0E0D0E02BC0CE01885A02
:1010500091094B97C0F7C85AD0E0CC0FDD1FC25E94
:10106000DC4F0990D881C02DD4641BC0D03490F4DB
:10107000D03208F0A8C0C83ED10598F0CE019150FA
:101080009F3108F78D2F6CDF082F8C2F90E0C5DE85
:10109000902B54C08C2F90E0C0DEDF70C82FD92B6E
:1010A000D06ACE01DF91CF911F910F910895C03882
:1010B00082E5D807B8F5C03682E5D80708F056C0F3
:1010C000C03482E5D807C8F4C03282E5D80708F0FA
:1010D00047C08C2F8695869520E2829FC0011124FF
:1010E000C37021E030E002C0220F331FCA95E2F73F
:1010F000E901C82BD92BDD68D4CF8C2F8695869536
:10110000877020E2829FC0011124C37021E030E08B
:1011100002C0220F331FCA95E2F7E901C82BD92B71
:10112000DC68BFCFC03C82E5D80750F48C2F8F71AC
:10113000C03AD24580F5982F84EF906AEC01B1CF88
:10114000CE01805C9245809708F07DCFDC2FDF7167
:10115000C0EFD06AA6CFA497D064A3CFD065A1CFAB
:101160008C2F8F71D82FC1EFD06A9BCF8C2F869593
:101170008695877020E2829FC0011124C37021E010
:1011800030E002C0220F331FCA95E2F7E901C82BF5
:10119000D92BDA6886CFE4DEC0E0D82FD06281CFC9
:1011A0008C2F8F71DDDE93E0CC0FDD1F9A95E1F778
:1011B000DF70282F84FF04C090E1899F90011124E3
:1011C000C22FD0696ECF8D2F8F71CADE082F8C2F62
:1011D00090E023DE902BEC01E1CF80E00895F894BD
:1011E000E82FE295EF70F0E041A18F7021E001C09F
:1011F000220F8A95EAF7922F9095942391A392A1BA
:10120000822F892B82A37894089581E080933307FD
:101210000895CF92DF92EF92FF921F93CF93DF93C7
:10122000462F172FE82FF0E0E25CF94F71110CC048
:10123000E4918E2F7E2F6E2FDF91CF911F91FF9023
:10124000EF90DF90CF900895F491EF2F86E0689FA4
:10125000E00111242FEF30E0CE01B9010E941533D7
:10126000DB01CA01880F991F65E56A9FA0016B9F8A
:10127000500D1124841B482F440F480FC901811BB6
:101280009109F89F7001F99FF00C11248F2D149F84
:10129000B0011124672F70E06901C61AD70AB601A0
:1012A000F69F6001F79FD00C1124A330B10549F1DE
:1012B000B901641B7109AB01149FB001159F700D3A
:1012C0001124672F70E0261B370BF29FA001F39FBC
:1012D000500D1124752FCC3FD34050F4A130B105EF
:1012E000A1F0129709F0A7CFEF2D852F7F2FA3CF65
:1012F000A430B10569F0169709F49DCF7F2D8D2D8F
:101300009ACF7D2DEF2D8F2F96CF7F2FED2D93CF61
:10131000E52F7F2DF8CF982F8091B607811529F002
:1013200081E0943208F080E0089581E09834FACFAB
:101330009C0180E090E0269F020E811D369F800D6B
:10134000911D1124830F911D089540911301509117
:10135000140125E038E0429FC001439F900D529F49
:10136000900D1124875E994C809313019093140182
:10137000890F0895982FE82F96FDE0958E2F8F7096
:1013800096FD8F5FE695E695E695E670F0E0E3530F
:10139000FD4F2181289F202D812D112422952F7012
:1013A0008295807F282B8081820F97FD81958058C0
:1013B00008951F93CF93DF93EB01182F822F86950B
:1013C000D9DF805887FD8195880F282F219F020E35
:1013D00020E0211D1124822FBE01DF91CF911F91AA
:1013E0000895622F0895E42FF0E0EE0FFF1FEB50F9
:1013F000FE4F6081621B08950F931F93022F50E0F0
:10140000FA01EE0FFF1FE754FE4FE5ADE052E7FD96
:10141000E195440F551F4B505E4FDA012C91201B74
:10142000310B2E0F620F1F910F9108950F931F9391
:10143000A02FB0E0FD01EE0FFF1FE754FE4F05ADFA
:101440000052110B2003F001219FF00D1124AA0F6F
:10145000BB1FAB50BE4F2C912057330B4203D00122
:10146000439FB00D11249F012A0F3B1F12F42158F6
:101470003F4F220F232F221F330B620F1F910F911B
:1014800008959091E904982B9093E9040895309180
:10149000B607311521F0843291052CF0089584327D
:1014A000910514F08497E2C308951F93CF93DF93BF
:1014B000C82FD0E0FE01EB57FD4F808190911101C4
:1014C000892389F042DF182F40DF20E8829FC00186
:1014D0001124792F7158612F809187079ADE472F49
:1014E000282FCE01D4DFDF91CF911F910895FF9275
:1014F0000F931F93CF93DF93182F062FF42EC0E086
:10150000D0E02F2D402F612FCE01C1DF2196C834AE
:10151000D105B9F7CDB7DEB7E5E00C945233982F7B
:10152000990F990F890F982F9B5F993408F098E4D1
:101530002091B607211104C0843228F484E2089572
:10154000953208F094E20895EF92FF920F931F9363
:10155000CF93DF937C0180911001E1DFC82F192F19
:10156000609188076695669521E0620F08F46FEF39
:101570008091E5049091E604DBDE082FD0E0812F16
:10158000C11730F0C8DECDB7DEB7E6E00C945133BA
:10159000FE01EB57FD4F808190911101892379F075
:1015A000609185077091860780918707202F4C2FC7
:1015B000F70109952EDE472F282FCE0168DF2196EF
:1015C000DECFA0E0B0E0E7EEFAE00C943333182F62
:1015D00080910F01811324C0909184079370209112
:1015E0000E0130E081E09217130609F480E0809349
:1015F00012018091890790911101981731F0809321
:10160000110140E060E080E072DF193058F4E12F12
:10161000E150E830E8F4F0E0EE51FC4C0C94733308
:1016200081E0E5CF1F3F09F43EC180E090911001B9
:101630009F5F9093100181115FC182E080930D0143
:1016400080911201811158C1111156C183E052C11C
:1016500080911201811549F340E060E080E047DFAE
:10166000E4CF809110015BDFC82F092F60918507BF
:101670007091860780918707CCDDF62EE72ED82E55
:10168000D0E00C1709F018F4802F45DECFCFFE0113
:10169000EB57FD4F808190911101892329F02D2D69
:1016A0004E2D6F2DCE01F3DE2196EBCF89ED99E023
:1016B0004BDFBCCF81EF99E0FBCF83EF99E0F8CF10
:1016C0008CEF99E0F5CF8091100129DFC82F092F09
:1016D0006091880766958091E5049091E60428DE84
:1016E000D82ED0E0CE01880F991F87549E4F7C01E1
:1016F0000C1751F248F2FE01EB57FD4F808190919B
:101700001101892309F44FC0F70144AD4057550B2F
:1017100085AD8052990B449F9001459F300D300D4F
:101720001124889FA001899F500D500D1124240F72
:10173000351F822F2230310520F19FEF213E8EE1AF
:10174000380740F4C901E5E096958795EA95E1F7F9
:10175000982F985F61E0462F490F5527551F5595E3
:101760004795842F449FF001459FF00DF00D112403
:101770002E173F07E8F4942F9150961760F7862FA5
:10178000815090E0BC01660F771F680F791F759537
:1017900067956D0D70918607809187073ADD472F19
:1017A000282FCE0174DE219682E0E80EF11CA0CF36
:1017B0004F3F39F3642F6F5FE0CF80911001AFDEB0
:1017C000C82FF92E60918807669566958091E5048B
:1017D0009091E604ADDDE82E805CCCDD8058D82EFB
:1017E0008E2DC8DD8058C82ED0E0CF1510F08F2D7B
:1017F0004CCFFE01EB57FD4F808190911101892361
:1018000079F06091850770918607809187070C2F8A
:101810002C2D4D2D0BDEFDDC472F282FCE0137DE82
:101820002196E3CFC0911001C1111DC060918807BE
:1018300020E1620F08F46FEF8091E5049091E604D7
:1018400077DD65E070E00E941533892B61F47DDD62
:1018500028E4829FA0011124852F880F880B5093C4
:101860000B0180930C018C2F5ADEEC019091120138
:10187000911115C020910B0130910C0128173105F1
:1018800080F02D17310568F4822F0FDE89E48093F4
:101890000B0110920C0105C08C2F07DECF5FCD1716
:1018A000D8F38D2FF2CE9091E604A091E704B09189
:1018B000E804892F9A2FAB2FA69597958795A69523
:1018C00097958795837090E0A0E0B0E08230910515
:1018D000A105B105B1F083309105A105B105A1F0D5
:1018E00040E060E010979040814081F464E180E046
:1018F000FEDD82E080930D01CDB7DEB7E8E00C9409
:101900004F3344E160E0F3CF44E164E184E1F0CFA0
:10191000CF93C82F811581F080911E0781110CC0D3
:1019200050DE10920F0180918407837080930E0126
:1019300063D583E080930D01C0931E07CF91089576
:101940009091840721E092279093840710920D01D3
:1019500098CD80918407837011F410920D018091CD
:1019600084078C7F81608093840708958091840729
:10197000837011F010920D01809184078C7F809309
:101980008407089590918407937091F0811589F0F0
:10199000893088F48F73880F880F982F20918407DF
:1019A0002370922B9093840710920D01862F69CD9E
:1019B000089581E0F0CF88E0EECF8091840786958E
:1019C00086958F5F893008F081E061E0DBCF809100
:1019D000840786958695815009F488E061E0D2CF2E
:1019E00090918407937059F08093850760938607E0
:1019F000493708F048E740938707822F42CD089582
:101A0000E4E8F7E0818190E021E04381628108967B
:101A1000E7CFE4E8F7E0818121E0438162818850EB
:101A2000990BDECFE4E8F7E0628120E1620F08F471
:101A30006FEF818121E0438190E0D2CFE4E8F7E0CD
:101A4000628120E1621B08F460E0818121E0438132
:101A500090E0C6CFE4E8F7E0438120E1420F08F4CC
:101A60004FEF818121E0628190E0BACFE4E8F7E0B6
:101A7000438120E1421B08F440E0818121E0628142
:101A800090E0AECF2091880730E1230F08F42FEFCC
:101A90002093880781E0F5CC2091880730E1231B53
:101AA00008F420E02093880781E0EBCCE0918907DF
:101AB000EF3F69F0E53069F0E23069F4EF5FF0E0A4
:101AC000EB54FE4F80818093890781E0DACCE0E01F
:101AD000F5CFE1E0F3CFE0E0F2CFE0918907EF3F0F
:101AE00091F0E53071F0E23019F0E1110EC0E3E061
:101AF000E150F0E0EB54FE4F80818093890781E054
:101B0000C0CCE1E0F5CFE3E0F4CFE0E0F2CF20910C
:101B1000F406382F3203C0011124923014F080E013
:101B200090E082519B4F8093EC049093ED040895D4
:101B30000F931F93CF93DF93A091EC04B091ED042A
:101B40009D012E5E3440620F731F613042E07407C6
:101B500010F060E072E04091EA045091EB04FC0167
:101B600001E010E02617370748F04093EA0450934D
:101B7000EB04DF91CF911F910F91089584919D9176
:101B8000981789F0ED018A93C901C5E0969587956C
:101B9000CA95E1F7E80102C0CC0FDD1F8A95E2F794
:101BA000CE014C2B592B2F5F3F4F3196DBCF9091BD
:101BB0007907292F30E070917A07A9014395437086
:101BC00050E07417150689F02958384F60FB87F9E3
:101BD000F90184839F5F93709093790780917707D1
:101BE0008F5F8093770781E0089580E0089590E00B
:101BF0006115D1F08A5E9E4FFC0180818F3F99F084
:101C0000E82FE295EF70F0E041A18F7021E001C074
:101C1000220F8A95EAF7922F9095942391A392A18F
:101C2000822F892B82A30895895E9E4FE5CF90E095
:101C30006115A9F08A5E9E4FFC0120812F3F91F033
:101C4000E22FE295EF70E05EF0E0808190E02F708F
:101C500002C0959587952A95E2F781700895895E6F
:101C60009E4FEACF80E00895539A0895FC01EE0F4D
:101C7000FF1FE80FF91FEA51FC4F61834083228365
:101C80000895FC01680F791F8FEF41E39191892737
:101C900028E030E0982F990F87FF09C0892F84270B
:101CA00021503040B9F7E617F70781F70895892FDB
:101CB000F7CF811144C0EFECF3E020E030E047E0E3
:101CC000429FC001439F900D1124DC01AC52BC4FD8
:101CD0005C9153FF06C05681511103C081539C4F44
:101CE00008952F5F3F4F37962330310549F761152F
:101CF00031F18091D40383FF1CC08091DB0383FF0B
:101D00001BC08091E20383FD1AC082E090E027E0CF
:101D1000289FF001299FF00D1124CF0181539C4F82
:101D2000DC0116961C92EC52FC4F20812860208327
:101D3000089580E090E0EBCF81E090E0E8CF80E094
:101D400090E008954115510511F0FA0109950895A3
:101D50008091B507811103C0809183070895E091B8
:101D6000DD07F091DE07309739F00190F081E02D2A
:101D7000309711F00995089580E00895A3E0B0E050
:101D8000E4ECFEE00C9439332091CD033091CE0386
:101D900028173907B1F08093CD039093CE03E091DB
:101DA000DD07F091DE07309761F00084F185E02DCA
:101DB000309739F023E029838A839B83CE010196F3
:101DC00009952396E2E00C945533A3E0B0E0EBEEE6
:101DD000FEE00C9439332091CB033091CC032817CB
:101DE0003907B1F08093CB039093CC03E091DD07EA
:101DF000F091DE07309761F00084F185E02D309797
:101E000039F024E029838A839B83CE0101960995CA
:101E10002396E2E00C94553390918E01913099F025
:101E2000AEE8B3E0EFEF90E02C91821759F01196F5
:101E3000EF3F19F4211101C0E92F9F5F9630A1F700
:101E4000EF3FC1F4089590910B0897FFE9CFE82F79
:101E5000E695E695E695803FA8F7F0E0EC56FC4F56
:101E6000877021E001C0220F8A95EAF78281822BD8
:101E700082830895FE2FFF0FFF0BE457FC4FF8CF2E
:101E800090918E01913021F490910B0897FD0CC038
:101E9000EEE8F3E09191891302C0DF011E9293E016
:101EA000E439F907B9F70895E82FE695E695E69540
:101EB000803FC8F7F0E0EC56FC4F9DEF81FD97EFB7
:101EC00080FF959582FD9295828189238283089572
:101ED00080918D0108952FB7F8946091C703709198
:101EE000C8038091C9039091CA032FBF08958091C0
:101EF000B507811539F0EFDF462F572FBC01CB0115
:101F0000BA010895E8DFDC01CB014091B707509199
:101F1000B8076091B9077091BA07480F591F6A1F37
:101F20007B1FEDCF87E797E7809300089093010828
:101F300088E19AE00FB6F894A895809360000FBEF0
:101F400090936000FFCF0895FC012091BD03309174
:101F5000BE032617370748F06115710529F49091E3
:101F6000E8009E779093E8009B0190E021153105F1
:101F700041F4911106C08091E80082FF32C080E0F8
:101F80000895809114078115C1F18530C1F18091C8
:101F9000E80083FD30C08091E80082FDECCF8091A5
:101FA000E80080FFE3CF8091F3004091F200582FCA
:101FB0002115310519F04830510558F091E04830AD
:101FC000510509F090E04091E8004E774093E80019
:101FD000CDCF81918093F100215031094F5F5F4F48
:101FE000E7CF80911407811541F0853041F0809151
:101FF000E80083FFC0CF81E0089582E0089583E088
:102000000895982F9093E900891771F07091EC0072
:102010002091ED005091F00021FD09C09F5F9730A5
:1020200089F78093E9000895762F242F50E03091AE
:10203000EB003E7F3093EB003091ED003D7F30931D
:10204000ED003091EB0031603093EB007093EC00C9
:102050002093ED005093F0002091EE0027FDDECF9D
:1020600008958091B70387FF13C08091E80082FF35
:1020700006C08091E8008B778093E80008958091F6
:1020800014078111F2CF0895809114078115D9F3B7
:102090008091E80080FFF8CF8091E8008E77ECCF48
:1020A0002091E4003091E50095E6A9012091EC0033
:1020B000822F817020FF06C08091E80080FF06C05B
:1020C00080E008952091E80022FD1AC08091140755
:1020D000811589F0853089F08091EB0085FD0FC076
:1020E0002091E4003091E50042175307F9F2915036
:1020F000E1F684E0089582E0089583E0089581E0A8
:102100000895CF93DF93C8EDD0E088818F7E8883D8
:10211000E7EDF0E080818160808384E082BF81E030
:102120008093B60388818E7F8883E2EE10821092BE
:10213000DA00A1EEB0E01C9288818F7788838881D5
:102140008068888388818F7D888319BC10921407EA
:102150001092B5031092F7061092B403A0EE8C9182
:102160008B7F8C9388818160888342E060E080E08F
:1021700048DFA1EEB0E08C918E7F8C93E2EEF0E030
:10218000808181608083808188608083E0EE8081AF
:102190008E7F8083888180618883DF91CF910895CD
:1021A000E8EDF0E080818E7F80831092E200109253
:1021B000DA001092E100A0EEB0E08C9181608C9387
:1021C00080818F77808319BCA7ED8C918E7F8C9353
:1021D00080818F7E80831092B6030895A0E0B0E0E6
:1021E000E4EFF0E10C942F33D82E80919A018D15F5
:1021F00049F000916108109162080115110539F448
:10220000D0929A01CDB7DEB7ECE00C944B338D2D14
:102210000E94EC05B82E9091600880E0891781F348
:10222000F8012081B21609F455C08F5F0B5F1F4F74
:10223000F5CFF8010180F281E02DEE0DFF1D208128
:10224000822F81568A31B8F420522052330B46E057
:10225000429FC001439F900D112425E0492D62E06B
:102260008057974F0E9486058FEFE81AF80A892D4C
:10227000865F982E65C0203240F720E2E6CFED124F
:102280000FC0A814B90401F580E698E020E14C2FB6
:1022900060E10E9486058FEFE81AF80AC85F6CC0FB
:1022A000C7010197A816B90691F080E398E0AE1433
:1022B000BF0461F31F3F29F080E198E0AE14BF0432
:1022C0002CF380E298E0E2CF80E598E0DFCF80E475
:1022D00098E0DCCF81819281892B09F491CFD09154
:1022E0005F08D11509F48CCFE3E6F8E080E491E0D3
:1022F00011920197E9F7F801A181B281FD010190E6
:102300000020E9F73197EA1BAE2ECD2EC3944AE0A8
:102310004E9F402D1124425080E590E09C01241BEB
:102320003109A90155954795942E2C2D220F220F86
:10233000220F821B910995958795C82FE12CF12CCE
:10234000EA1408F476CFEFE4F8E010E0A081B18160
:10235000109719F08C918B1529F032961F5F1D1381
:10236000F5CF1FEFE12CF12CA12EB12EBB0CBB0839
:102370008D2F8150990B4C01EC1408F041CFE110E6
:102380007ECF80E898E0111509F480CF80E798E0CF
:102390007DCFA0E0B0E0EFECF1E10C9431337C01B3
:1023A0006B015A01809198070AE010E08A3010F022
:1023B00001E010E0C1E0D0E0B601C701F5010995E8
:1023C000811115C021960C171D078CF0CC9F900130
:1023D000CD9F300D300D112480E090E045E34A950B
:1023E000F1F70000019682179307C1F7E5CFCDB74B
:1023F000DEB7EAE00C944D333BB1377F2BB1286058
:102400004FB7F89486EE93E0FC010196508168E0A6
:102410002BB9000000C057FF3BB9550F000000C0AA
:1024200000C000C03BB900C06A9591F754E08E3BF4
:10243000950751F74FBF8FE594E00197F1F700C082
:10244000000008950F931F93CF93DF93EB018A0150
:1024500090911407943059F58093E9008FEF909193
:10246000E80095FD06C095ED9A95F1F700008150C2
:10247000B1F78091E80085FF1AC012DE811112C009
:102480008091E80085FD06C08091E8008E778093FA
:10249000E800F3CF88818093F1000150104011F0E3
:1024A0002196EECF8091E8008E778093E800DF914F
:1024B000CF911F910F910895603229F440E250E0CE
:1024C000BC0182E0BFCF0895CF93DF93EC0148E0D9
:1024D00050E0BC0181E0B6DF88E0FE01AFEBB3E085
:1024E00001900D928A95E1F7DF91CF91089540E236
:1024F00050E0BC0184E0A6CF43E050E0BC0184E0A2
:10250000A1CF90910C0892FB222720F9281779F08F
:1025100080FB92F990930C0860910B0870910C0865
:1025200084E090E00E94DC3382E00C94C8060895B9
:102530001F93CF93DF93122F8630E0F46A30D0F4EC
:102540004630C0F4C42FD0E0CC0FDD1F2CE0629FDA
:10255000C00DD11D112498E7899FC00DD11D1124F4
:10256000632FCE0189960E94C233612FCE018A96D5
:102570000E94C233DF91CF911F910895AF92BF9215
:10258000CF92DF92FF920F931F93CF93DF93A12CF3
:10259000B12CC0E06501D0E018C021E030E0C430CB
:1025A00020F4F801859195919C014F2D6D2F8C2F72
:1025B000BFDFF3940E5F1F4F8F2D863071F7DF5F03
:1025C00086E0C80ED11CDA3039F08601000F111FE9
:1025D000065E1D4FF12CE1CFCF5F8CE3A80EB11C3E
:1025E000C630C1F6DF91CF911F910F91FF90DF9020
:1025F000CF90BF90AF90089580918E01813069F5A2
:1026000080910B0887FF29C00E94DE068093950306
:1026100040E250E06DEB77E084E993E00E94803384
:10262000892BD1F080E2E4E9F3E0ADEBB7E0019073
:102630000D928A95E1F7E091DD07F091DE07309782
:1026400059F00480F581E02D309731F086E08093D9
:10265000940384E993E0099508950E94DE0680932F
:102660008C0348E050E06FED77E08CE893E00E9447
:102670008033892B89F388E0ECE8F3E0AFEDB7E035
:1026800001900D928A95E1F7E091DD07F091DE0768
:10269000309711F30280F381E02D3097E9F28CE856
:1026A00093E0D9CF811531F090910508982B909344
:1026B0000508A2CF0895811531F090910D08982B4F
:1026C00090930D0899CF0895811519F00E94050780
:1026D00093CF0895811539F0809590910D08892345
:1026E00080930D0889CF0895CF93C82F8115C1F02D
:1026F0008450813A70F580918E01813021F480916F
:102700000B0887FD0FC0EEE8F3E08081C817E9F001
:10271000319683E0E439F807C1F78C2F7DDB6CDF5D
:10272000CF910895EC2FE695E695E695F0E0EC560E
:10273000FC4F828190E04C2F477021E001C0220FB6
:102740004A95EAF78223892B41F38C2F99DB54DFDA
:10275000E4CF8C2F805E883060F4C77081E001C0C8
:10276000880FCA95EAF7C0910508C82BC0930508E1
:10277000D6CF8C2F855A833028F48C2F8452990B16
:10278000FDDACECFC85ACB3158F6EC2FF0E0EE0F81
:10279000FF1FEC5AFC4F8081918117DBC1CFCF9393
:1027A000DF93EC01805E9109089720F06BE573E1FF
:1027B000209711F462E573E1CE010E94CF058C2FC2
:1027C00093DFDF91CF910895CF93DF93EC018A815E
:1027D000823039F4FB0182819381E1DF8D81826057
:1027E0008D83DF91CF910895FB0180819181D7CFB7
:1027F000811511F1982F9450913A10F441DBFCCEE1
:10280000982F905E983058F4982F81E091FD84E0E5
:1028100090FD880F92FD82950E940507F0CF982FBA
:10282000955A933018F480E090E0A8CA885A8B310A
:1028300018F480E090E0C9CA0895CF93DF93EC01CB
:10284000D7DFCE01805E9109089720F06AE673E138
:10285000209711F464E673E1CE010E94CF05DF9169
:10286000CF910895FC018281813059F48FE39CE976
:102870000197F1F700C00000FB0180819181DDCF5D
:1028800008958230E9F7FB0182819381F8CF1F938D
:10289000CF93DF93182FC0E5D0E0893311F0CAE061
:1028A000D0E0812F21DF8FE99FE00197F1F700C091
:1028B00000002197C1F7812F9BDFDF91CF911F91FE
:1028C000089580E090917A0720917907291711F1F6
:1028D000E92FF0E0E558F84F8081282F2F779F5F90
:1028E000937090937A07909178079F5F9093780701
:1028F000211531F0213041F487FF0AC08EE403C076
:1029000087FF04C08AEAC3DF81E0DCCF89EAFBCF1E
:102910008BE4F9CF08951092050880918E018130E3
:1029200099F480910B0887FF0FC0E6E9F3E08EE190
:1029300011928A95E9F780E090E020DA80E090E05B
:1029400044DA10920D0858CEEEE8F3E086E0F0CFBE
:10295000E2DF88E19AE00FB6F894A89580936000D2
:102960000FBE90936000FFCFAAE2B0E0EAEBF4E183
:102970000C94383387EB93E0FC0101962091F10031
:10298000208323E08F3B9207B9F78091B803893009
:1029900009F457C0C8F4823009F4B3C0833009F495
:1029A00083C0813081F18091E80083FFE7C080918E
:1029B000B7039091B8039A3008F0E0C0E92FF0E037
:1029C000E651FC4C0C9473338A3009F48AC08B3086
:1029D00051F78091B703813231F78091BB03909119
:1029E000BC03892B01F78091E800877F8093E80082
:1029F00038DB81E09091B903911101C080E08093B0
:102A00008E0189DFD0CF8091B703813A61F6809142
:102A1000E800877F8093E8008091BB039091BC031E
:102A2000892B59F060E080E090E070E08DDA8091D1
:102A3000E8008B778093E800B6CF68E08FEB93E0F7
:102A4000F4CF8091B703813209F0ADCF8091BB0301
:102A50009091BC038D7F892B09F0A5CF8091E80070
:102A6000877F8093E8008091E80082FF18C0209162
:102A7000F3008091F200922F029731F48091F100DF
:102A8000813011F0863021F48091F10080938D0126
:102A90008091E8008B778093E800E3DA84CF80911F
:102AA00014078111E0CF7FCF8091B703813A09F0FD
:102AB0007ACF8091BB039091BC03892B09F073CF2F
:102AC0008091E800877F8093E8008091E80080FF94
:102AD000FCCF80918E018093F1008091E8008E7789
:102AE000DACF8091B703813209F05DCF8091E800A1
:102AF000877F8093E800B5DA8091BA0380938C01D8
:102B000052CF8091B703813A09F04DCF8091E80010
:102B1000877F8093E8008091E80080FFFCCF809160
:102B20008C01D9CF803889F0823841F58091BB0380
:102B30008F70873018F58093E9008091EB0085FB5A
:102B4000882780F91092E90006C08091F706880F67
:102B50009091B403892B9091E800977F9093E800BF
:102B60008093F1001092F1008091E8008E7723C0ED
:102B7000811116C08091B903813009F18091E8007C
:102B800083FF0AC08091E800877F8093E8008091EE
:102B9000EB0080628093EB00AA96E3E00C94543340
:102BA000823061F78091B903811579F01092E900C4
:102BB0008091E800877F8093E80053DADFCF93307D
:102BC00009F080E08093F706F1CF8091BB038F700E
:102BD000282F2150263090F68093E9002091EB00B9
:102BE00020FFE4CF933031F48091EB00806280933A
:102BF000EB00DCCF9091EB0090619093EB0021E033
:102C000001C0220F8A95EAF72093EA001092EA00A9
:102C10008091EB008860EBCF8111B0CF8091B90338
:102C20008F77182F8091E3008078812B8093E300C9
:102C30008091E800877F8093E80013DA8091E800B4
:102C400080FFFCCF8091E30080688093E30083E005
:102C5000111101C082E08093140790CF8058823018
:102C600008F08CCF8091B9039091BA038C3D23E09A
:102C7000920789F583E08A838AE289834FB7F894C3
:102C8000DE01139620E03EE051E2E32FF0E05093A6
:102C90005700849120FF03C082958F703F5F8F7033
:102CA0008A30B8F0895C8D931D922F5F243169F7CB
:102CB0004FBF8091E800877F8093E8006AE270E070
:102CC000CE01019641D98091E8008B778093E8008E
:102CD00055CF805DE8CF292F30E02330310509F44E
:102CE0004DC078F52130310509F47CC08BE590E0CA
:102CF000EFE7F1E02230310509F040CF2091E80004
:102D0000277F2093E8002091BD033091BE038217F6
:102D1000930708F49C0140E02115310509F067C0D4
:102D2000411165C08091E80082FDCDCF80911407EC
:102D3000811549F2853039F28091E80083FFF2CFA6
:102D4000C2CF8091BB039091BC0321323105D9F1F0
:102D50002232310509F012CF8330910508F00ECFF1
:102D6000FC01EE0FFF1FEF55FE4F0190F081E02DAB
:102D700082569E4FDC018C9190E011C0282F30E0EC
:102D8000813089F022303105B1F0232B09F0F6CEE5
:102D9000E6E1F2E0E4918E2F90E0E6E1F2E00097C8
:102DA00009F4ECCEABCFEAEFF1E0E4918E2F90E0A6
:102DB000EAEFF1E0F4CFECEEF1E0E4918E2F90E059
:102DC000ECEEF1E0ECCF8330910508F0D7CE880F20
:102DD000991FFC01E955FE4F0190F081E02D89E03B
:102DE00090E08CCF82E190E0EAEDF1E087CF809136
:102DF0001407811509F467CF853009F464CF8091F9
:102E0000E80083FD60CF8091E80082FD8BCF809148
:102E1000E80080FF81CF4091F3008091F200942F71
:102E20002115310519F08830910550F041E00897DF
:102E300009F040E08091E8008E778093E8006CCF45
:102E400044914093F1003196215031090196E8CF29
:102E5000803809F093CE8091E800877F8093E80066
:102E60008091B5038093F1007FCE811187CE809150
:102E7000B903182F823008F081CE8091E800877F57
:102E80008093E8001093B503ECD81115D9F084E0D5
:102E90008093140742E061EC81E0B3D842E261EC38
:102EA00084E0AFD842E261EC82E0ABD842E260EC71
:102EB00083E0A7D880911407843051F482E0809396
:102EC0008F015CCE8091E30087FDE1CF81E0E0CF10
:102ED00081E0F5CFCF93DF93EB01FC014481558175
:102EE00060857185CE010E94A20E9B819095809194
:102EF0000D08892380930D088C810E9405077CDBD7
:102F000087E019928A95E9F7DF91CF9108950F93A1
:102F10001F93CF93DF938C01EB018D8181FD17C04F
:102F200082608D8380910D089B81892B80930D0891
:102F3000809105089C81892B809305085DDBF80151
:102F40004281538160857185CE010E94A20E10924C
:102F5000FF07109200088D8180FD03C0BE01C801EB
:102F6000B9DFDF91CF911F910F910895CF92DF923A
:102F7000FF920F931F93CF93DF936901E801082F0E
:102F8000880F110B41155105B1F0F80133E0EE0F38
:102F9000FF1F3A95E1F7EC5DFE4F818192818A5BDC
:102FA000984FE0812E2F30E04E17510508F49A011A
:102FB000A9010E948D33C8010E94A732F82E811505
:102FC000E1F02097D1F0C80123E0880F991F2A95DE
:102FD000E1F7FC01EC5DFE4F2381422F50E0C21768
:102FE000D10508F4AE018C5D9E4FFC0164817581B2
:102FF0006A5B784FC6010E948D338F2DDF91CF9190
:103000001F910F91FF90DF90CF900895A4E0B0E062
:10301000ECE0F8E10C943533E0902F07F0903007A6
:1030200000913107109132070E946B0FDC01CB0138
:103030008E199F09A00BB10B11E084369105A105F3
:10304000B10510F10E94770FDC01CB010296A11DA2
:10305000B11D89839A83AB83BC8300E010E09801A3
:1030600044E050E0BE016F5F7F4F86E07FDF182FA6
:10307000811551F00E946B0F60932F0770933007FA
:103080008093310790933207812F2496E6E00C94C9
:103090005133A1E0B0E0EFE4F8E10C942933662E5F
:1030A0002A01190168018D019E012F5F3F4F40E009
:1030B00050E0BA015BDF182F8115B1F1F201808079
:1030C0009180A280B3800E946B0F79806819790982
:1030D0008A099B09643671058105910530F4B701B1
:1030E000C6010E94410E8715F9F08701910140E069
:1030F00050E0BA01862D3ADF082FB701C6010E94C1
:10310000410E10E087110BC0102F117000FF07C097
:103110000E946B0FF2016083718382839383812FFE
:103120002196E2E10C944533A701B601C1010E944A
:103130008D33F5CFA5E0B0E0E0EAF8E10C9433334D
:103140006B017D0107E417E0CE0101969C0142E48A
:1031500057E061E080E09DDF811559F095E09E0128
:103160002F5F3F4FF901ADE3B7E001900D929A95C3
:10317000E1F795E0EDE3F7E0D60101900D929A9525
:10318000E1F72596E8E00C944F33A8E0B0E0EBECD3
:10319000F8E10C9435337D0102E517E09E012F5FC5
:1031A0003F4F45E357E064E083E073DF182F81155C
:1031B00099F19091510780913407981769F1909196
:1031C000550780915407891709F1E92FF0E0E65B74
:1031D000F84F848587FB662760F99F5F9370909313
:1031E0005507909153079F5F909353078F770E94E5
:1031F000D70DF82E8111E3CF00E010E09801A8016F
:10320000B80185E0B3DEF8221F2D02C0F110F4CF23
:103210008091510780933407812F2896E6E00C9423
:103220005133A0E0B0E0E7E1F9E10C942F33D82E60
:10323000EB01C42E59014801E880F9800A811B8105
:103240000E946B0FDC01CB018E199F09A00BB10B03
:1032500084369105A105B10510F4C11479F000E0A0
:1032600010E09801A401B5018D2D80DE811539F0A3
:103270000E946B0F688379838A839B8381E0CDB73B
:10328000DEB7ECE00C944B330F931F9341E0909129
:103290005E0780910908981301C040E001E010E04A
:1032A00029E038E06BE277E087E0BBDF811571F061
:1032B00041E090915F0780910808981301C040E0B9
:1032C00028E038E067E277E088E0ABDF1F910F91FC
:1032D0000895A1E0B0E0EFE6F9E10C943733809176
:1032E0001907898320916A0790E041E028171906A1
:1032F00009F440E08D019E012F5F3F4F6AE177E0C6
:103300008BE08FDF2196E4E00C945333CF92DF9271
:10331000FF920F931F93CF93DF93F82E6B01EA0177
:10332000A801B901CE010E94803341E0892B09F444
:1033300040E09E01B6018F2D74DFDF91CF911F9188
:103340000F91FF90DF90CF9008950F931F9305E0AA
:1033500010E02CE437E0AC0169E377E082E0D6DFEF
:103360001F910F910895A1E0B0E0E9EBF9E10C9411
:1033700037330E94A80E898301E010E020E637E091
:10338000AE014F5F5F4F63E277E089E0BFDF2196D8
:10339000E4E00C945333A9E0B0E0E1EDF9E10C94E2
:1033A000373388E0E4E8F7E09E012F5F3F4FD90113
:1033B00001900D928A95E1F780911E07898709E0B7
:1033C00010E021E637E0CE010196AC016FE177E035
:1033D0008AE09CDF2996E4E00C945333ACE0B0E043
:1033E000E4EFF9E10C9437338091940790919507BD
:1033F000A0919607B091970789839A83AB83BC838A
:103400008091900790919107A0919207B0919307B6
:103410008D839E83AF83B88780918C0790918D07B1
:10342000A0918E07B0918F0789879A87AB87BC8759
:103430000CE010E02BE637E0AE014F5F5F4F65E137
:1034400077E08CE063DF2C96E4E00C9453330F9329
:103450001F93CF93DF93863008F56A30F8F4463037
:10346000E8F4C42FD0E0CC0FDD1F9CE0699FC00DB5
:10347000D11D112498E7899FC00DD11D1124CE01C3
:1034800089960E94A633082FCE018A960E94A63301
:10349000902FDF91CF911F910F91089580E090E0E0
:1034A000F8CF462F7A3030F4663020F4863010F4AE
:1034B000672FCDCF80E090E00895CF92DF92FF920A
:1034C0000F931F93CF93DF936C01009109088091B4
:1034D0000808082BC5E0D0E010E0C8010C2E02C09F
:1034E000959587950A94E2F780FD0CC02197A8F77F
:1034F000F12C8F2DDF91CF911F910F91FF90DF90D5
:10350000CF900895FC2EB6018C2FCBDF0E940108CE
:10351000019761F3EECF1F93CF93DF93FC012581D9
:10352000C081D181CE01211579F0611569F0C5DF27
:10353000182F682FCE010E941806BE01812FB1DF1F
:10354000DF91CF911F9108950E944E06182FF5CF5D
:10355000CF93DF93EC01B1DFBE01A3DF0E9401082E
:10356000DF91CF910895FC012481211599F080818C
:103570009181EEDF282F92959F70963099F060F43C
:10358000925F9F70923030F4203FB1F038F481E0C8
:10359000283E38F080E008959A5FF3CF81E0243F21
:1035A000C9F7089591E0213F09F090E081E0283EBD
:1035B00008F080E0892B089581E00895673021E0CC
:1035C00072078105910528F4CB0187509D4F0C941B
:1035D000A63380E00895CF92DF92EF92FF92CF93CF
:1035E000DF93EC01C880D980EA80FB80B601C70177
:1035F000E5DF9FEFC91AD90AE90AF90AC882D98218
:10360000EA82FB82DF91CF91FF90EF90DF90CF9025
:10361000089585E290E00E94A633863269F486E23E
:1036200090E00E94A633863039F487E290E00E9451
:10363000A63391E0863109F090E0892F81700895DA
:1036400080E090E00E94AE33833E9E4F09F4E1CFCC
:1036500080E0089548E050E067E170E084E897E09A
:103660000E94B3331092E904089581E180938407A6
:1036700080919B0190919C01A0919D018093850771
:1036800090938607A09387078FE7809388078FEF33
:1036900080938907DFCFCF92DF92EF92FF920E9453
:1036A000770FAB01BC014093E0045093E104809399
:1036B000E2047093E3048091E40490910D01923050
:1036C00049F1F0F4911123C0109210014093E504E8
:1036D0005093E6046093E7047093E80480911E071A
:1036E000811108C080918407982F937019F08695F6
:1036F0008695982F9093E40481E080930D0102C099
:10370000933099F0FF90EF90DF90CF9008950E9452
:10371000E10AF8CF80930F01809184078370809332
:103720000E010E94FC1183E0E8CF8091E904811131
:1037300091DFC090E504D090E604E090E704F090BB
:10374000E8048091B507811571F00E946B0F6C1928
:103750007D098E099F09653071058105910590F2FB
:1037600010920D01CFCF0E94770FF1CFA0E1B0E012
:10377000ECEBFBE10C942B33FE013196DF0180E191
:103780001D928A95E9F701E110E099EFA92E92E0E8
:10379000B92E612C712C230153944A189E2E8F2E22
:1037A0006201730181E148165104610471041CF047
:1037B00080E1C82ED12CA601B501892D982D0E943B
:1037C000B333AC0CBD1C0D2C000C00084C185D086C
:1037D000600870080150104019F76096E0E10C9401
:1037E00047336FEF85E290E00E94C2336FEF86E2CD
:1037F00090E00E94C2336FEF87E290E00E94C233F4
:1038000060E088E290E00E94C2330E94BE12AEDF08
:1038100066E285E290E00E94C23366E086E290E0D4
:103820000E94C23366E187E290E00C94C23363EEFB
:103830007EEF80E090E00E94DC3360E082E090E088
:103840000E94C23381E08093080861E083E090E049
:103850000E94C23360E074E184E090E00E94DC33B7
:1038600004DFBFDF60E070E0AB018FE090E00E941A
:10387000D43360E070E0AB0183E190E00E94D43388
:10388000E9CEAB0124E630E0BC0188E70E94DE30DF
:103890009C0181E0232B09F080E008958091EF06E0
:1038A0008115F1F00E946B0FDC01CB01805A95412C
:1038B000AF4FBF4F8093F0069093F106A093F206AE
:1038C000B093F3068091190781110AC062E070E09D
:1038D0008CE396E0D6DF811519F081E0809319071B
:1038E00008958091EF06811561F080911907811587
:1038F00041F062E070E08AE396E0C3DF811110924C
:10390000190708951F921FB61F9211248F939F933A
:10391000AF93BF938091F606811113C08091C703C6
:103920009091C803A091C903B091CA034196A11D0B
:10393000B11D8093C7039093C803A093C903B093AC
:10394000CA03BF91AF919F918F911F901FBE1F908F
:1039500018952FB7F8948091C7039091C803A09150
:10396000C903B091CA032FBF0895CF93DF93EC0131
:10397000F0DF8C1B9D0BDF91CF910895AFE0B0E09D
:10398000E4ECFCE10C943033FE013196DF018AE077
:103990001D928A95E9F783E1C82E83E0D82E7F0136
:1039A000AE2E9F2C0EE113E0F60181916F018F3F47
:1039B00009F43DC0F894E82FE295EF70F0E021A102
:1039C0008F7041E001C0440F8A95EAF7922F942B43
:1039D00091A392A1842F8095892382A3789400C01B
:1039E000E8E1F3E031E0B12C21912F3F79F0A22FF3
:1039F000A295AF70A05EB0E08C9190E02F7002C0F5
:103A0000959587952A95E2F780FFB7C080E0B82AA0
:103A1000330F0E171F0741F7F60182918F3F11F008
:103A20000E94EF0880EA8A95F1F7F701B0828FEFE4
:103A3000E81AF80A88E1C81683E0D80609F0B4CF7E
:103A40004AE050E06A2D792D8BEA97E00E9480339E
:103A5000009749F02AE0EA2DF92DABEAB7E0019092
:103A60000D922A95E1F70091AA0710E00056184F31
:103A7000892B09F484C081E080939F076ADF8093DB
:103A80009D0790939E078091B507811509F4CEC0DC
:103A90007E018BE0E80EF11CF70185E011928A951A
:103AA000E9F7809198078A3008F08CC04AE958E11C
:103AB000B701C8010E94C911811509F4A6C045EAE1
:103AC00059E1B701C8010E94C911811509F49DC0CF
:103AD00045EC58E1B701C8010E94C911811509F4EC
:103AE00094C046E058E1B701C8010E94C911811590
:103AF00009F48BC044E459E1B701C8010E94C9111F
:103B0000811509F482C043EB59E1B701C8010E9455
:103B1000C911811509F479C04BEC59E1B701C8010D
:103B20000E94C911811509F470C049E659E1B70135
:103B3000C8010E94C911811509F467C04EEE59E110
:103B4000B701C8010E94C911811509F45EC0109225
:103B5000980780919C0790E045E050E0B7018056BF
:103B6000984F0E94803321E020939B07892B09F016
:103B70003FC02F96EBE00C944C33832F48CF8091BD
:103B80009F07811509F47FCFE0909D07F0909E0775
:103B9000E0DE8E199F09059708F475CF45E050E0E7
:103BA0006BEA77E0C8010E948033892B41F085E001
:103BB000EBEAF7E0D80101900D928A95E1F71092B7
:103BC0009F0761CFC0909907D0909A07C2DE8C19E9
:103BD0009D09843F914008F069CF80919B07811532
:103BE00041F2F70185E011928A95E9F710929B075F
:103BF000A0919C07B0E0A056B84F85E0FE013B962F
:103C000001900D928A95E1F7B4CF809198078F3F8C
:103C100031F49FDE8093990790939A07DECF8F5FF0
:103C2000809398078A3008F494CFF3CFE0909C07F4
:103C3000F12CC7018056984F7C0185E0F801A7E47C
:103C4000B7E001900D928A95E1F765E070E087E4B6
:103C500097E00E94410E8093460785E0ECE4F7E090
:103C6000D70101900D928A95E1F788E0E7E7F7E048
:103C7000A2E5B7E001900D928A95E1F768E070E067
:103C800082E597E00E94410E80935107C0905A0749
:103C9000D0905B07E0905C07F0905D0780917F0714
:103CA00090918007A0918107B0918207C816D9062C
:103CB000EA06FB06B1F0C0927F07D0928007E0923F
:103CC0008107F09282070E946B0FC61AD70AE80A92
:103CD000F90AC092B707D092B807E092B907F092FC
:103CE000BA0780915E078093090880915F078093EF
:103CF0000808809160078093830788E0E1E6F7E099
:103D0000A4E8B7E001900D928A95E1F780916907E8
:103D10000E94880C80916A07811591F1BFDD809126
:103D2000730790917407A0917507B0917607409141
:103D30006F07509170076091710770917207009141
:103D40006B0710916C0720916D0730916E070093FF
:103D50009407109395072093960730939707409305
:103D60009007509391076093920770939307809305
:103D70008C0790938D07A0938E07B0938F07F9CE91
:103D8000B0DDCDCF2F923F924F925F926F927F9294
:103D90009F92AF92BF92CF92DF92EF92FF920F93DA
:103DA0001F93CF93DF938091EF06811509F47BC0B9
:103DB000C091DE04D091DF04CCDD8C1B9D0B81977C
:103DC00008F450C0C6DD8093DE049093DF0480E0E9
:103DD0000E94870D809109080E94EE108091B6071D
:103DE000811509F48DC080E00E94870D60E670E0C7
:103DF0008AE595E00E94980D83E00E94870DE0918E
:103E0000EC04F091ED049F012E5E3440BF016E5A28
:103E10007340613082E0780710F060E072E040911A
:103E2000EA045091EB04A3E6B8E0D1E0ED2EF12CCA
:103E30002617370708F449C04093EA045093EB046F
:103E40008DE00E94870D60E470E08AEF95E00E94AB
:103E5000980D8FE00E94870D60E270E08AEF93E09A
:103E60000E94980D8091EA049091EB04892B09F04F
:103E700068C0809119078115B1F00E946B0FC09145
:103E8000F006D091F106E091F206F091F306DC0124
:103E9000CB018C1B9D0BAE0BBF0B8F3F9F4FAF4FCA
:103EA000BF4708F41EDDDF91CF911F910F91FF9066
:103EB000EF90DF90CF90BF90AF909F907F906F90EA
:103EC0005F904F903F902F9008958D919191891719
:103ED000A1F08F0101501109E8018883C901C5E0F3
:103EE00096958795CA95E1F7E70102C0CC0FDD1FD3
:103EF0008A95E2F7CE014C2B592B2F5F3F4F98CF7D
:103F00000E94A80ECAEBD4E081FD02C0CAE1D4E051
:103F100080E00E94870D60E670E08AE595E00E94EF
:103F2000980D84E00E94870D60EA70E0CE010E9447
:103F3000980D8DE00E94870D60E470E08AEB95E0BB
:103F40008FCF8091EF06811509F493CF8091EE0613
:103F500081118FCFA3DCC0E0D1E12091EA04309140
:103F6000EB042115310509F484CFD15009F481CF38
:103F700041E050E001C0CF5F8C2F90E07A010C2E21
:103F800002C0EE0CFF1C0A94E2F7B7016223732310
:103F9000672B89F32091F50620FD43C09695879500
:103FA00096958795482F282F9C2F9295990F90765C
:103FB000392F315E842F909306018093090130934D
:103FC000070120930A0124E630E047E050E064E076
:103FD00071E088E70E949430892B09F04ACF80E293
:103FE000C89FA00111248091F50680FD23C0425195
:103FF0005B4F04E610E020E230E060E488E70E94D6
:104000002431892B09F035CFE094F0948091EA04B3
:104010009091EB04E822F922E092EA04F092EB049A
:104020009CCF9C2F990F990F990F392F395F80E002
:1040300023E0C1CFEEEBF4E080E211928A95E9F73C
:1040400031EB632E31E0732E0DEA11E065EB71E088
:10405000D301ED913D01D8018D918D01282F240FC1
:10406000352F311D1901F0E0E254FB4F80E090E064
:1040700027E0A22EA81ABB24B394082E01C0BB0CC3
:104080000A94EAF7910122513B4F2901C12CD20138
:10409000DD902D01DB202A2D2C19277030E0AD2D6D
:1040A000022E01C0AA0F0A94EAF79A2E31952195A3
:1040B00031092770332701C0D6942A95EAF79D2845
:1040C0002081922A9082C3942C2D283001F70196EA
:1040D00031968830910561F66615770509F0B8CFFD
:1040E00004E610E020E24EEB54E087CFFF920F93FE
:1040F0001F93CF93DF93C62FD42FF22E8115A9F0F3
:104100006093030826DC8093E4039093E50381E049
:10411000C1FD84E0C0FD880FC2FD82950E9452134C
:10412000CDB7DEB7E5E00C945233809103086813F5
:1041300031C00091E4031091E5030BDC801B910B6F
:10414000883C910538F51D2F105ECD17A1F0C77082
:1041500001E0802F01C0880FCA95EAF70E9464131E
:10416000183048F48D2F877001C0000F8A95EAF748
:10417000802F0E9452138F2D0E94471481E0D1FDA1
:1041800084E0D0FD880FD2FD8295183048F60E9459
:104190006413C6CF81E0C1FD84E0C0FD880FC2FD7D
:1041A0008295F5CFA4E0B0E0E8EDF0E20C942E3378
:1041B0007C01FC018481811509F421C161E0C70102
:1041C000AAD96C01F70185818115D1F00091FF0713
:1041D000109100080115110599F0C016D10689F05B
:1041E00020E9A22E21E0B22E011511F0A12CB12C54
:1041F00060E0802F0E94590EFC01892B09F048C015
:104200008601F701958102348EE7180709F499C0F9
:1042100008F04EC000348EE7180709F458C0013486
:104220008EE7180709F472C0F7018581811509F43A
:104230006FC1980137572038310508F069C1003146
:1042400008F0CEC066E071E080E090E0B7D981115F
:10425000C7C0A12CB12C4501011184C089829A826A
:10426000AB82BC828E010F5F1F4FC801B4D9B02E44
:10427000A12E813008F4B4C009F0DCC0C801ABD96C
:10428000813009F082C0C801A6D90E94471483C0BA
:10429000858184608583C082D182BF01C5010E946F
:1042A000871710920D0861E0C70135D98C01A9CF9D
:1042B00003348EE7180709F0B7CF80910C0881709E
:1042C000911509F44BC081112FC08DE40DC0809170
:1042D0000C088170911569F0811549F084E00E9405
:1042E000B0070E94521380E50E9474139DCF81E0B5
:1042F000F6CF811549F084E00E94B0070E94641354
:1043000080E50E94F81390CF81E0F6CF80910C08F1
:104310008170911559F0811539F084E00E94B00741
:104320000E9452138FE4E0CF81E0F8CF811539F07D
:1043300084E00E94B0070E9464138FE4E2CF81E022
:10434000F8CF80910C088170911521F08111CFCFA9
:104350008AE4CACF8111D8CF8AE4D3CF8111EFCFBD
:104360008DE4CFCF87E0881681E09806A104B104E0
:10437000B9F1B401C50122D99FEF891A990AA90A96
:10438000B90A8111EFCF015067CF823059F4C801CB
:1043900022D90E9474138FE39CE90197F1F700C0C2
:1043A000000063CF833029F4C80115D90E94F813A7
:1043B000F2CF843069F4C8010ED9C12CD12C282F3A
:1043C0002053330B2A303105F0F0C114D10441F5EC
:1043D000EFE3FCE93197F1F700C00000811145CF10
:1043E00080910A08877059F0F7018581811539F0AD
:1043F00080910C0882FF03C082E00E94C8062496C8
:10440000EDE00C944A334AE04C9DC0014D9D900D67
:104410001124280F391F69018B2D9A2DDCD8CFCF9D
:10442000EFE9FFE03197F1F700C0000091E0C91A11
:10443000D108CBCFE82FF0E0E057F84F9491792ED8
:10444000282F26952695269530E0F901E058F84F5B
:10445000C4908770D12C082E02C0D594C7940A94BA
:10446000E2F7F901E059F84FA490B12C082E02C0F0
:10447000B594A7940A94E2F7205A384FF901849032
:10448000912C02C0959487948A95E2F7C0FE09C0EA
:1044900081EE0E9474138FE39CE90197F1F700C04D
:1044A0000000A0FE09C086EE0E9474138FE39CE911
:1044B0000197F1F700C00000872D0E9474138FE36D
:1044C0009CE90197F1F700C00000872D0E94F813C6
:1044D0008FE39CE90197F1F700C00000A0FE09C03E
:1044E00086EE0E94F8138FE39CE90197F1F700C074
:1044F0000000C0FE09C081EE0E94F8138FE39CE922
:104500000197F1F700C0000080FEAFCE8CE2BDCE77
:10451000312F375509F07EC0A02EB12C011160CF8C
:10452000682F80E00E94590E6C01892B09F458CF46
:10453000F7018581F601958180FB90F995838115BE
:1045400009F448C006DA8093010890930208F60146
:1045500082818F5F828380910D0890910508892B5D
:10456000838380910608848340919001509191014A
:104570006091980170919901C6010E94A20EF60106
:10458000858181FD03C0A12C97E5B92EA092FF077C
:10459000B0920008F7019581911509F450C410926A
:1045A0000308980130572332310508F035C484E000
:1045B00090E00E94AE3380930B0890930C08F801B2
:1045C000E150F047E232F10508F04BC0EC50FC4CF2
:1045D0000C9473334091960150919701609198012A
:1045E00070919901C6010E94A20EF601858181FF9A
:1045F000D1CFB60180E991E00E946A178091FF0750
:10460000909100088115974529F61092FF071092A6
:104610000008C0CFF801E851FC47E730F10508F089
:10462000B9CFEA5EFB4C0C94733326E241EE61EEA7
:104630005DDDD6CE27E245EE65EEFACF26E241EE0D
:1046400060EEF6CF27E245EE64EEF2CF26E241EED1
:1046500062EEEECF27E245EE66EEEACF28E241E0D9
:10466000EBCF80910B08816080930B0860910B0861
:1046700070910C0884E090E00E94DC330E948B145F
:10468000AFCE80910C08886080930C08EFCF8091AA
:104690000B088260E9CF80910B088460E5CF8091A0
:1046A0000B088860E1CF80910C088160EDCF80918C
:1046B0000C088260E9CF80910B088061D5CF809192
:1046C0000B088062D1CF80910B088064CDCF0E940F
:1046D0008B1480910B088068C7CF80910B088C6089
:1046E000C3CF80910C088360CFCF80910B088E7F61
:1046F000BBCF80910C08877FC7CF80910B088D7F3F
:10470000B3CF80910B088B7FAFCF80910B08877F51
:10471000ABCF80910C088E7FB7CF80910C088D7F36
:10472000B3CF80910B088F7E9FCF80910B088F7D38
:104730009BCF80910B088F7B97CF0E948B14809129
:104740000B088F7791CF80910B08837F8DCF80915D
:104750000C088C7F99CF90910B08892F8B7F92FF4B
:104760008460877F92FF88607FCF80910C08982FAC
:10477000909590FB80F990FB81F986CF90910B0882
:10478000892F8F7B96FF80646FCF0E948B1490914E
:104790000B08892F97FB87F9805866CF61E08EE080
:1047A00090E00E94C23362CF60E0F9CF90910B0895
:1047B000892F8F7E94FF806157CF90910B08892FAE
:1047C0008E7F90FF816050CF90910C08892F877F5A
:1047D00093FF886059CF8A7A91E0811101C090E0FF
:1047E00090930408811106C089E20E940C0F0E9478
:1047F000FC12F6CD85E3F9CF85E32BC381E00E945F
:10480000A00CEECD811579F10E94E70CE9CD811560
:1048100079F10E94090DE4CD811579F10E941E0DF8
:10482000DFCD811579F10E94360DDACD811579F150
:104830000E944C0DD5CD809105088272F801E0549C
:10484000F847EF30F10580F5E35EFB4C0C947333D1
:104850000E94A90C81E00E94410AC2CD0E94B60CC0
:10486000F9CF811589F20E94DD0CBACD811589F24C
:104870000E94000DB5CD811589F20E94120DB0CDB8
:10488000811589F20E942A0DABCD811589F20E9413
:10489000420DA6CD811529F00E946D0DA1CD811587
:1048A000D9F30E94560D9CCD07378CE71807F1F01D
:1048B00008378CE7180729F19801205E324520322D
:1048C000310520F5911134C00F7181E090E002C0F4
:1048D000880F991F0A95E2F78C01682F83E090E01A
:1048E0000E94C233802F0E94FE057ACD81E091158F
:1048F00051F00E94040643E062E081E00E948106DC
:104900006FCD82E0F4CF0E940D06F5CF911581F1B5
:104910000B358CE7180711F10C358CE7180799F067
:104920000A358CE71807C1F001308CE71807F1F061
:1049300003308CE71807A1F001151C47C9F40E9449
:104940008B140E94920F80910C08002482FF039424
:10495000802D0E94811244CD81E0FBCF80E0F9CF11
:104960006FEF7FEF80E090E00E94DC330E94A8149C
:10497000F70100811181911509F45BC0C8010E9403
:104980005D1AD82E682FC8010E941806B8018D2D17
:104990000E94511A0E940108182FA92EF701B58014
:1049A000D680D2948FE0D82280910A08877001F1D6
:1049B000CB2CB114F1F0892F807F803461F0812FEE
:1049C000805E8830A8F0892F807E803221F41230FA
:1049D00078F0D11469F080910C0882FF09C082E060
:1049E0000E94C80680910A088770CC24C394811164
:1049F000C12C8A2D82958F70883009F40EC1C0F5C4
:104A00008430E0F4823008F444C00A2D0F708A2DFF
:104A1000807F803211F00295007F113008F472C05F
:104A200009F4BBC0B11409F4C6C0D11409F488C09C
:104A300048C0C8010E944E06D82EA8CF09F4D1C0A4
:104A4000C11409F419C180910A0880FD15C1F7014C
:104A500015828695869586950E940406C701A2DB7D
:104A600080910A088695869586950E940D0604C158
:104A7000893009F44DC18A5F8F70823008F7123F88
:104A800009F058C18A2D8F71B11051C10E940406DE
:104A9000F1C00A2D0F708A2D803110F00295007F31
:104AA000B114B9F0011569F0812F805E883010F0E3
:104AB000111109C080910508802B809305080E9480
:104AC000FC12812F2FC080910D08802B80930D0840
:104AD000F6CF812F0E94F813011509F4B1CF812F71
:104AE000805E883010F0111104C0802F0E940507ED
:104AF00006C0009580910D08802380930D080E94C8
:104B0000FC129ECF80910C0882FD16C0B11469F092
:104B1000011539F080910508802B809305080E94CB
:104B2000FC1280E00E9474138BCF80E00E94F81387
:104B3000011509F485CFD9CFB114A9F0D11004C063
:104B4000802F0E9452137CCF8D2D813009F078CFB9
:104B500080910608902F9823091709F471CF802BB4
:104B6000809306086DCFD1106BCF802F0E94641305
:104B700090910608802F892329F0802F8095892322
:104B80008093060880910708902F982309F458CF46
:104B9000009508230093070853CF8D2DB11421F001
:104BA000863008F04DCFCCCF853008F049CF802F2C
:104BB0000E94641345CFD114D1F3193369F48FEFF8
:104BC00097EE23E0815090402040E1F700C00000C4
:104BD000812F0E94F81334CF8FE39CE90197F1F7FE
:104BE000F5CF8A2D869586958370813060F009F027
:104BF00027CF812F9A2D9370B11002C080E090E0F2
:104C00000E94E50E1DCF812F9A2D9370B11002C026
:104C100080E090E00E94BE0E13CF8A2D8370E1F5F4
:104C2000B11028C0812F829586958770880F880FD4
:104C3000412F4F70082E01C0440F0A94EAF7212F2C
:104C4000207114FF06C02FE001C0220F8A95EAF7F9
:104C500020958A2D869586958370982F8230A1F0B5
:104C60008330B9F080910808913059F0242B8223C9
:104C70000E94FE050E94A80E60E0C7010E948B1AE8
:104C8000BECB842B822BF4CF242B80910808822763
:104C9000EFCF822F842BECCFB11459F1A0FEEACFD5
:104CA000812F829586958770880F880F412F4F70CE
:104CB000082E01C0440F0A94EAF7212F207114FF37
:104CC00006C02FE001C0220F8A95EAF720958A2DB1
:104CD000869586958370982F823091F08330A9F065
:104CE00080910908913049F0242B82230E9401060B
:104CF000C1CF823008F4BECFD3CF842B822BF6CF26
:104D0000242B809109088227F1CF822F842BEECFAC
:104D10008A2D8F70082FB11431F00E940406812F64
:104D20000E945213A7CF812F0E946413802F0E94EC
:104D30000D06A0CF70F4103FC9F0113F91F0B114EF
:104D400009F451C0D11409F44BC0812F0E9474138F
:104D500091CF133FF9F0143F91F790910C0892FD19
:104D600026C08A2D8F71B11411F390CE8D2DB11400
:104D700079F0853008F07ECF8A2D8F71282F81E061
:104D800001C0880F2A95EAF7909109088927AECFCC
:104D90008630F0CF80E0B11409F4A8CF8A2D8F714E
:104DA000982F81E001C0880F9A95EAF79FCFB11440
:104DB00061F08A2D8F7192FF69CE982F990F990F0C
:104DC000990F936090930A0861CE81E00E94C80613
:104DD0008D2D823008F44ECF82E00E94C8064ACF63
:104DE0008A2D8F7153CED114A1F0193369F48FEF4E
:104DF00097EE23E0815090402040E1F700C0000092
:104E0000812F0E94F81336CF8FE39CE90197F1F7C9
:104E1000F5CF8A2D8F718BCF8091050806312CE755
:104E2000120709F4D8CC8272F801E052F847EB304F
:104E3000F10508F039CDE45DFB4C0C947333063179
:104E40008CE7180709F0F7CC809104088111D4CCC5
:104E500089E20E94400FCBCC80914E08803170F4E3
:104E600080914D08811551F0E0910F0820910E08B6
:104E700030914908409148082E1301C00895BF01A0
:104E800087E0E89FF0011124DF01A05FB74F14967F
:104E90008C911497811551F111968C911197831370
:104EA00025C08C91841322C015968C911597811181
:104EB0001DC012968D919D91A0914A08B0914B080A
:104EC0008A1B9B0B883C910588F480914E088F705B
:104ED000806180934E08EA5EF74F80818F70806119
:104EE000808388E498E05ED90C94BE066F5F7F4FA4
:104EF000FB01E770C1CFADE0B0E0E1E8F7E20C9470
:104F00002E338C0186E0F801DE01189601900D9297
:104F10008A95E1F7F801F580848198E4892E98E07C
:104F2000992E70904C08711017C0811591F0F114F2
:104F300009F40EC1C8010E94B31A811509F408C111
:104F400087E0F801A8E4B8E001900D928A95E1F7B6
:104F500083DFFF24F39455C0D080A280B380C0903B
:104F60004D0820914A0830914B08A501421B530B74
:104F7000C11409F4BDC0483C510508F076C0811544
:104F800041F3809149089180E0904E089E2D903128
:104F900008F057C0981214C0809148088D1110C0B5
:104FA000F11049C08E2D8F70806180934E0888E487
:104FB00098E0F8D880914E08F8018683F12C21C042
:104FC000F11039C040E0692D8D2D0E949F0640E010
:104FD000692D8D2D0E949F06F82E8111EFCF8885B7
:104FE00099850E94A81A292F22952F70903470F469
:104FF0009F70223098F09115A9F0F80196819031B8
:1050000088F48F2D2D96EDE00C944A332A5F2F7093
:10501000223060F0C801C6D8FC2CF3CF911511F0F6
:10502000811579F3805E883060F3F4CF803F48F3D8
:10503000815F8330F9CF80914E08816080934E0864
:10504000BDCF981237C0809148088D1133C0F11040
:1050500031C0E682C801A6D887E0F801A8E4B8E02C
:1050600001900D928A95E1F774CFE0904E089E2D45
:10507000903148F488E498E095D8F40187E01192E3
:105080008A95E9F79BCF811509F463CF9091490880
:10509000818198130FC0809148088D110BC0F110C9
:1050A00009C0E682C8017ED8F40187E011928A9592
:1050B000E9F74FCFC8010E94B31A811509F448C01F
:1050C000F11409F445C08E2D803208F439CF809157
:1050D00048089091490889839A83AB82BC827D827B
:1050E0001E8280914E088F83CE0101965BD828CF17
:1050F000483C510508F0C1CF811509F42ACFF114BD
:1051000039F1909149088181981318C0809148081D
:105110008D1114C080914E0880FD9ECF803108F41F
:105120009BCF8683807F803F09F494CF8681982F20
:10513000907F905F8F70892B86838CCFC8010E94EF
:10514000B31A8111FDCE80914E08816080934E0884
:10515000C80128D8FECEABE1B0E0E1EBF8E20C9458
:1051600037334E8B5F8B688F798F8A8F192F9B8F88
:10517000911110920D081D8A86E0FE017696DE01DF
:105180001F9601900D928A95E1F70A8D011561F045
:105190000B8B1C8B61E0CE010F960E948B1A61E095
:1051A000CE010F960E948B1A0B8B1C8B87E0FE01A1
:1051B0003F96DE01189601900D928A95E1F7CE0197
:1051C000089699DE81112EC020910E0830910F08AB
:1051D00087E0AE01485F5F4FFA0147505109DA019D
:1051E00001900D928A95E1F78C858115D9F0822F77
:1051F00090E08395877090E0AC0134171506E1F0DC
:1052000097E0929FD0011124A05FB74F9E012F5FBE
:105210003F4FF90101900D929A95E1F740930E08E6
:105220000E94BE0680910F0890910E08891311C04C
:105230006B96E4E00C9453330E948B1410920E088A
:1052400010920F08E8E4F8E087E011928A95E9F7F8
:10525000E9CF27E0829FC0011124805F974F4BDE8A
:10526000811531F380910F08909110080196877095
:1052700080930F08D7CFA6E0B0E0E1E4F9E20C9408
:1052800037330E94A91C8C018091BB079091BC0709
:105290008017910771F019821A820E94A91CBC0123
:1052A00049815A8180E090E056DF0093BB0710935C
:1052B000BC072696E4E00C945333CDB7DEB7A09735
:1052C0000FB6F894DEBF0FBECDBF85B7806885BF2F
:1052D00085B7806885BF84B7877F84BF0FB6F89491
:1052E000A8958091600088618093600010926000B2
:1052F0000FBE80E890E00FB6F89480936100909321
:1053000061000FBE81E080938F018DEE98E0809365
:105310008A0390938B030E94D0100E948110809189
:10532000E20084608093E2007894809114078115F4
:1053300099F08091E9001091EC008F7010FB11271B
:1053400017F9182B1092E9008091E80083FD0E9464
:10535000B4141F701093E90082E084BD93E095BD02
:105360009AEF97BD80936E001092B7071092B8071E
:105370001092B9071092BA070E94091B811102C04E
:105380000E94F11B8091D80080618093D8008AE14F
:105390008A95F1F700C08091D900182F117080FD17
:1053A00004C00E94D010109214071093B5070E94F9
:1053B000201B811102C00E94171C8EE090E00E9409
:1053C000A633811529F060E08EE090E00E94C233A0
:1053D0008EE090E00E94A63391E0811101C090E040
:1053E0009093B607909315018091B5078111CED7A0
:1053F000E7E7F7E088E011928A95E9F78091B60730
:1054000091E0282F292720930F07909312078111ED
:1054100006C084EF8093170185EF8093160160E04A
:1054200080E00E94F70D61E080E00E94F70D8FE8B8
:1054300091E00197F1F700C0000010E080911207A1
:10544000181708F462C08091B60790E0811101C07E
:1054500095E09093AA0785E0891B80939C0703E160
:1054600013E0F80181918F018F3F11F00E94EF0846
:1054700083E008311807A9F778E1E72E73E0F72EEB
:105480000EE113E0F70181917F018F3F11F00E943F
:10549000EF080E151F05B1F7E0EAF7E08AE0119278
:1054A0008A95E9F7EBEAF7E08AE011928A95E9F745
:1054B0000E94201B811102C00E94171C82E090E014
:1054C0000E94A6338093020784E090E00E94AE33EE
:1054D00080930B0890930C080E94BE1C8FEF96E7F8
:1054E00021E0815090402040E1F700C000000E9480
:1054F000BE1C8091A00780FF1AC06FEF7FEF80E095
:1055000090E00E94DC330E94920F60E0812F0E94A5
:10551000170E082F61E0812F0E94170EE12FF0E097
:10552000E05FF84F880F802B80831F5F87CF83E079
:1055300090E00E94A6330E94FE050E94340E81E096
:105540008093E90448E050E067E170E084E897E088
:105550000E9496331092E90480918407843010F4FD
:105560000E94351B83E08093F50680E28093F40669
:10557000A8D56BE070E085E597E00E94411C81159D
:10558000E9F18091F50665E070E081FD06C180E5F6
:1055900097E00E94411C811589F16DE070E08EE377
:1055A00097E00E94411C811549F10E946B0FDC01BC
:1055B000CB01805A9541AF4FBF4F8093F006909337
:1055C000F106A093F206B093F306EEEEF4E0DF01ED
:1055D00080E092E01D920197E9F7E093EC04F093EC
:1055E000ED048FEF9FEF8093EA049093EB0481E04A
:1055F0008093EF06809319071092EE068091B5070D
:10560000811101C0C6D68DEE92E08093610890931F
:10561000620884E080936008ADEEB2E020E013966B
:105620008C911397811501F12830F0F4822F90E0CE
:10563000FC01EE0FFF1FE15BF74F8F01009761F058
:10564000F801529142918F01FA01348114966C91C4
:105650001497631708F4A4C0880F991F815B974FB4
:10566000FC01A083B1832F5F159683E0A130B807BA
:10567000B1F620935F08809109080E94EE1088E13E
:1056800091E08093DD079093DE0741E0A42EB12CDA
:105690008091140700E110E432E1F32E853009F423
:1056A000DFC00E94BE1C23E0C22E27E0D22E80EA7B
:1056B00097E01C01FC01D6019D91808127E0AD306F
:1056C000B20709F4DAC031969817B1F34090B507E4
:1056D00098EFE92E96E0F92E912CF10181901F01AF
:1056E000F60181916F01881509F442C08825582E72
:1056F00000E010E077247394852D872189F1682CD0
:1057000067204114F9F0F701808190E09501002EA7
:1057100001C0220F0A94EAF78223892B99F40983A6
:105720009A820E94A91C8B839C8381E08D8391E0E7
:10573000611001C090E09E8349815A816B817C8118
:105740008D8109DD61100CC08A2D002E01C0880FEB
:105750000A94EAF7982F9095F70180818923808336
:10576000770C0F5F1F4F0630110531F6F60182925C
:1057700093948FEFE81AF80A892D8A3009F0ADCF9B
:105780000E94770F60939407709395078093960714
:1057900090939707DD24D39474C08BE497E0F9CEFF
:1057A0000197F8014283538349CF809114078430D5
:1057B00051F10E944B1B81E00E94880C0E94711CD9
:1057C0001092F60688E190E00FB6F894A8958093C1
:1057D00060000FBE1093600083B7817F846083BF39
:1057E00083B7816083BF7894889583B78E7F83BFAA
:1057F0000FB6F894A895809160008861809360004E
:10580000109260000FBE0E94BE1CE0EAF7E0A8EF15
:10581000B6E080E021912D9391E0211101C090E04C
:10582000892B97E0EA3AF907A9F78115C9F0809129
:10583000F7068115A9F009BDF9BC09B400FEFDCF3A
:105840008091D8008F7D8093D8008091E0008260A5
:105850008093E0008091E00081FDFCCF0E948B14DA
:1058600080911407853009F4A0CF0E948B140E9408
:10587000A80E80E00E94880C14CF981327CFFBDC81
:10588000D12C8091B507811531F1E090FF07F090A0
:105890000008E114F104F9F00091010810910208E8
:1058A0000E94A91C801B910B893C9105A0F000E986
:1058B00011E0E11411F000E010E060E08E2D0E9494
:1058C000590E009741F0FC01258122FD04C0BC0166
:1058D000C8010E9487170E944B1B1091B507111534
:1058E00019F00E946114182F80913307811551F02F
:1058F000109233078091790780937A078091770718
:105900008093780700E039C061E0802F0E94170E75
:10591000F82E60E0802F0E94170EFF0C8F29202F99
:1059200030E0D901A05FB84FEC919E2F937089179A
:1059300019F1EE0FEE0FE82BEC9380910F07800F1B
:10594000EF70F0E0EF5FFC4F235F384F7901C080CC
:10595000F9019081C90E9C2D60E092301CF49F3FAC
:105960001CF461E00E94D70D8C2DCC0C990B62E0E9
:1059700070E0A6D6F70180830F5F809112070817A9
:1059800018F28091B507811519F00E946114182B47
:10599000111579F00E94770F60939007709391072B
:1059A00080939207909393070E94C21E0E944E1C00
:1059B00004C00E94C21ED110F9CF0E94A80E90917F
:1059C0001307891721F0809313070E946B0F8091B2
:1059D0001407843009F05CCE83E08093E900809165
:1059E000E80082FF55CE8091E80090E085FF05C079
:1059F0000E945010811591F091E08091E8008B7722
:105A00008093E800911509F443CE8981E82FE15095
:105A1000E33168F5F0E0E95CFB4C65C680E2E82E16
:105A2000F12C8E010F5F1F4F8091E80085FD0AC0A9
:105A30008091E8008B778093E8000E9450108115D8
:105A400099F3DACF8091F100F801808381E0E81AC0
:105A5000F10891F2E7CF1A828CE08B8319C08A811A
:105A6000833081F138F4813029F1823051F08FEFA9
:105A700089830EC08430D9F71B821C821D821E824E
:105A800007C088E290E062D61B821C821D828E8352
:105A9000E091DD07F091DE07309709F4F9CD02843B
:105AA000F385E02D309709F4F3CD60E2CE01019645
:105AB0000995EECD0E946B0F1CD66B837C838D8382
:105AC0009E83E6CF8B8190E0FE0134968A3091056B
:105AD000FCF611920196FACF8A81823031F085303E
:105AE00031F680E00E94A00CD3CF6B817C818D8148
:105AF0009E81FFD588E290E045D6CACF4C816B816C
:105B00008A810E94271A9827892798278D839E8348
:105B1000BFCF2D813E813227232732274C816B81D5
:105B20008A810E949812B4CF0E94BE12B1CF9A818E
:105B3000933009F09CCF883009F439C0893009F4DA
:105B400062C08B81833061F158F4813091F08230F2
:105B500009F09ECF8C8181111CC00E94B60C98CF99
:105B6000843009F095CF8C8120E0409187076D81CA
:105B70000CC04C8128E7429F040E40E0411D1124D7
:105B80008091850720E06091860790E00E94F00CEC
:105B90007FCF0E94A90C60E08C810E94C20C78CF5C
:105BA0008C818093880780E00E94410A71CF8B81AD
:105BB000833031F170F48130B1F0823009F068CF78
:105BC00080918407982F9370C9F0869586958C8371
:105BD0005FCF843009F05CCF809185078C83809102
:105BE00086078D8355CF809187072FEF829FC00155
:105BF000112468E770E019D56C834ACF80E0E7CFC5
:105C000080918807E4CF0E942A1B42CF80E18A83DB
:105C10003FCF81E08A8387E020CF4A805B80542495
:105C200045245424612C712C8E010F5F1F4FEC8092
:105C3000E00EF12EF11C0E151F0509F429CF87E0A7
:105C4000481681E058066104710470F4C20187505F
:105C50009D4F7CD5F80184830F5F1F4F8FEF481A4B
:105C6000580A680A780AE7CF80E0F4CF9C80CA809F
:105C7000DB80DC24CD24DC24E12CF12C8E010F5FB1
:105C80001F4F27013201491451046104710408F0C7
:105C9000FFCE87E0C81681E0D806E104F10430F4B5
:105CA000F8016481C60187509D4F6CD58FEF481A6B
:105CB000580A680A780A8FEFC81AD80AE80AF80A58
:105CC0000F5F1F4FE0CF0E94B61BE2CE86E09FCF52
:105CD0009C80CA80DB80DC24CD24DC24E12CF12CE8
:105CE000270132018E010B5F1F4F491451046104DB
:105CF000710408F0CDCE80EDC81682E0D806E1042C
:105D0000F10488F4C601899621D5F80181938F01A9
:105D10008FEF481A580A680A780A8FEFC81AD80A0B
:105D2000E80AF80AE2CF80E0F0CF9C80CA80DB80EE
:105D3000DC24CD24DC24E12CF12C8E010F5F1F4FDD
:105D400027013201491451046104710408F0A0CE06
:105D500080EDC81682E0D806E104F10428F4F801C9
:105D60006481C60189960ED58FEF481A580A680AD1
:105D7000780A8FEFC81AD80AE80AF80A0F5F1F4F8F
:105D8000E1CF78941F921FB61F9211248F939F9397
:105D9000AF93BF938091C7039091C803A091C903AB
:105DA000B091CA030196A11DB11D8093C7039093C2
:105DB000C803A093C903B093CA03BF91AF919F9149
:105DC0008F911F901FBE1F9018951F920F920FB6B4
:105DD0000F9211242F933F934F935F936F937F9371
:105DE0008F939F93AF93BF93EF93FF938091E100C5
:105DF00082FF09C08091E20082FF05C08091E1002E
:105E00008B7F8093E1008091DA0080FF24C0809135
:105E1000D80080FF20C08091DA008E7F8093DA0066
:105E20008091D90080FFA9C080E189BD82E189BD50
:105E300009B400FEFDCF81E0809314078091B60382
:105E4000811109C00E94D0100E9481108091E2004F
:105E500084608093E2008091E10080FF1AC080910D
:105E6000E20080FF16C08091E2008E7F8093E20006
:105E70008091E20080618093E2008091D80080628E
:105E80008093D80019BC85E08093140783E0809349
:105E90008F018091E10084FF2FC08091E20084FF98
:105EA0002BC080E189BD82E189BD09B400FEFDCF30
:105EB0008091D8008F7D8093D8008091E1008F7E03
:105EC0008093E1008091E2008F7E8093E2008091D8
:105ED000E20081608093E2008091B503811509F4AE
:105EE00052C084E08093140780911407843009F035
:105EF00052C082E080938F018091E10083FF2CC02B
:105F00008091E20083FF28C08091E100877F809329
:105F1000E10082E0809314071092B5038091E100C4
:105F20008E7F8093E1008091E2008E7F8093E2007B
:105F30008091E20080618093E20042E060E080E0D6
:105F40000E9401108091F00088608093F00081E051
:105F500080938F0180938E01FF91EF91BF91AF915C
:105F60009F918F917F916F915F914F913F912F9171
:105F70000F900FBE0F901F90189519BC1092140728
:105F80001092B60368CF8091E30087FF02C083E0E0
:105F9000A9CF81E0A7CF81E0ADCF1F920F920FB6BE
:105FA0000F9211241F932F933F934F935F936F93FF
:105FB0007F938F939F93AF93BF93CF93DF93EF9391
:105FC000FF93E9EEF0E080811091EC008F7010FB00
:105FD000112717F9182B1082C0EFD0E08881877F36
:105FE000888378940E94B414E9EEF0E010828881EE
:105FF000886088831F701083FF91EF91DF91CF91AC
:10600000BF91AF919F918F917F916F915F914F91D0
:106010003F912F911F910F900FBE0F901F901895D9
:10602000EF92FF921F93CF93DF93182FEB01109203
:10603000BC0084EA8093BC000E94A91C7C01809172
:10604000BC0087FF26C08091B900887F883029F086
:106050008091B900887F803189F51093BB0084E876
:106060008093BC000E94A91C7C018091BC0087FF2A
:106070001EC02091B900287F80E090E0283189F08F
:1060800081E090E0203409F480E0919581959109B8
:1060900008C0C7010E94B51CC817D90780F68EEF4B
:1060A0009FEFDF91CF911F91FF90EF900895C7016F
:1060B0000E94B51CC817D907C0F6F1CF8FEF9FEF2C
:1060C000F0CF1092B9008CE08093B80008950F9340
:1060D0001F93CF93DF93EB018093BB0084E8809301
:1060E000BC000E94A91C8C018091BC0087FF10C0DD
:1060F0002091B900287F81E090E0283209F480E007
:10610000919581959109DF91CF911F910F910895FC
:10611000CF3FDC0749F3C8010E94B51CC817D90757
:1061200018F78EEF9FEFEFCFA0E0B0E0E9E9F0E3E2
:1061300095C2982E862E772E6A0179010E94A91C9D
:106140005C0184E1E816F10410F18FEFE816FE041B
:1061500009F1C70164E170E068D2162F072F612FA3
:10616000702F892D5DDFEC01892BB1F4082D172DDF
:10617000C00ED11E0C151D0511F02097C1F084E949
:106180008093BC00CE01CDB7DEB7EDE083C211E055
:1061900000E0E5CF15E0FCCF8FEFE816FE04F9F242
:1061A000C5010E94B51CE816F906C8F6DFCFB70195
:1061B000F80181918F018BDFEC01DCCFA0E0B0E032
:1061C000E3EEF0E34BC2982E862E772E6A0189010A
:1061D0000E94A91C5C010431110500F10F3F10075A
:1061E00001F1C80164E170E020D2EB01BE01892D0C
:1061F00017DF7C01892BB9F4C82DD72DCC0EDD1EFD
:10620000CC15DD0519F0E114F104B9F084E98093AF
:10621000BC00C701CDB7DEB7EDE03CC2C1E0D0E0C5
:10622000E5CFC5E0FCCF0F3F100701F3C5010E9489
:10623000B51C08171907D0F6DFCFFE018491B8010D
:1062400046DF7C012196DCCFA0E0B0E0E9E2F1E39B
:1062500004C2982E862E742E652E6901E8010E94D4
:10626000A91C5C010431110508F10F3F100711F161
:10627000C80164E170E0D9D1F62EE72E6F2D7E2D96
:10628000892DCEDE8C01892BC1F0CF3FDC07B1F325
:10629000C5010E94B51CC817D90780F784E980930F
:1062A000BC00C801CDB7DEB7EEE0F3C1FF24F39424
:1062B000E12CE4CF85E0F82EFBCFBE01882D07DF6F
:1062C0008C01E72CF62CCE0CDF1CEC14FD0431F312
:1062D0000115110519F7BE01F70181917F01F7DE64
:1062E0008C01F3CF8EE14A9B02C08150E1F74A9BBB
:1062F000FECF08955A9880E28A95F1F75A9A089548
:10630000FC018BE08A95F1F728E080E090E031E035
:1063100040E14A95F1F7880F4A9B02C081609327BC
:1063200042E04A95F1F7000040E14A95F1F721502B
:1063300079F720E12A95F1F729B132E03A95F1F7A2
:10634000000030E13A95F1F731E022FD93272081FA
:10635000920F90830895A1E0B0E0E0EBF1E385C1F6
:1063600019828C017C01E60EF11CBCDFCE01019686
:10637000C7DFF80181938F01EE15FF05B1F781E0CA
:106380009981911180E02196E6E08BC1529A5A9A48
:10639000089552985A9AEA9AE9E6F0E080818F7C53
:1063A000808308956150770B91E001C0990F6A9541
:1063B000EAF7692F90E021E0611108C0911591F092
:1063C0005A9A80E28A95F1F75A980895362F382321
:1063D00039F05A9A922730E23A95F1F76695ECCF68
:1063E0005A98F9CF5A98EDCFFF920F931F93CF93FE
:1063F000DF93EC018C01060F111D8991F82E7ADFD5
:1064000068E08F2DCFDFC017D107B9F7CDB7DEB762
:10641000E5E048C11F920F920FB60F9211240F931F
:106420001F932F933F934F935F936F937F938F931C
:106430009F93AF93BF93EF93FF93CF93DF930F920D
:10644000CDB7DEB719824EDFCE01019659DF082F96
:10645000069506950695282F22952570902F957004
:10646000920F292F237096959695920F98279770E3
:106470008981892B09F055C00E3008F052C080E1A7
:106480008A95F1F75A9A529A82E08A95F1F700C0FC
:106490005A9888E0089F80011124D801AC5DBE4F56
:1064A0001696ED91FD911897309791F06091110338
:1064B0007091120314962D913D91260F371F159759
:1064C0008D919D91680F791F4C9113978C9109952F
:1064D000F801EC5DFE4F6381611549F020911103D5
:1064E0003091120384819581820F931F7DDF02DF3B
:1064F00080E18A95F1F75A9852985A9A80E18A95E4
:10650000F1F7F801EC5DFE4F6081611549F02091D3
:1065100011033091120381819281820F931F1BDF3F
:10652000E1DE0F90DF91CF91FF91EF91BF91AF919D
:106530009F918F917F916F915F914F913F912F919B
:106540001F910F910F900FBE0F901F9018950F93F2
:106550001F93CF93DF93EC010E970CF05EC0F8947D
:10656000529A5A9885E08A95F1F700009C2F9695EB
:1065700095708C2F8570980F892F837096959695BE
:10658000292F93E0CC0FDD1F9A95E1F7280F822F7A
:106590008C2B082FAFDE00C068E0802F03DF80E186
:1065A0008A95F1F752985A9A4A9B30C087E090E05A
:1065B0004A992EC0FE01EC5DFE4F6381611559F0D2
:1065C000209111033091120384819581820F931FD2
:1065D000C2DE8115F9F086DE80E28A95F1F75A98DD
:1065E000529A80E18A95F1F7CC5DDE4F68816115A2
:1065F00049F0209111033091120389819A81820F11
:10660000931FF2DE77DE789481E008C000C0CCCF23
:10661000019749F4529A5A9A789480E0DF91CF9189
:106620001F910F91089500C0C3CFAA1BBB1B51E15E
:1066300007C0AA1FBB1FA617B70710F0A61BB70BF2
:10664000881F991F5A95A9F780959095BC01CD0197
:1066500008952F923F924F925F926F927F928F9206
:106660009F92AF92BF92CF92DF92EF92FF920F93E1
:106670001F93CF93DF93CDB7DEB7CA1BDB0B0FB6EB
:10668000F894DEBF0FBECDBF09942A8839884888A8
:106690005F846E847D848C849B84AA84B984C8843E
:1066A000DF80EE80FD800C811B81AA81B981CE0F35
:1066B000D11D0FB6F894DEBF0FBECDBFED0108951A
:1066C00097FB072E16F4009406D077FD08D0ADDFB7
:1066D00007FC05D03EF4909581959F4F08957095E5
:1066E00061957F4F0895EE0FFF1F0590F491E02D07
:1066F0000994692796276927782787277827089597
:10670000FB01DC0104C08D910190801921F44150FE
:106710005040C8F7881B990B0895FB01DC0102C0AB
:1067200001900D9241505040D8F70895DC01CB0103
:10673000FC01F999FECF06C0F2BDE1BDF89A319691
:1067400000B40D9241505040B8F70895F999FECF2A
:1067500092BD81BDF89A992780B50895A8E1B0E06F
:1067600042E050E0E5CFDC01A40FB51F415050409E
:1067700040F0CB01840F951F2E9105D04150504021
:10678000D8F70895262FF999FECF92BD81BDF89ACA
:10679000019700B4021639F01FBA20BD0FB6F89465
:1067A000FA9AF99A0FBE08950396272FECDFEADFD5
:1067B000252FE9DF242FE7CF0196272FE4DFE2CF53
:1067C000F894FFCF310B560B5A0B5D0B600B630B2C
:1067D000DD0B120C9215B815BE15B815BE150C16AA
:1067E0002E16BE15281735177523DD237D23472365
:1067F0004B2381234F23852391235B23D6235F23C0
:10680000952363239923BE2367239D23C5236D23EB
:10681000A323AB235323892357238D237123A7233A
:10682000B523CE23D42341237923E4231E2322231B
:1068300015231A2326232A232E2328242E24FE233D
:1068400002243124072436240C243B241124402420
:10685000162445244A244F24FE23022431240724ED
:1068600036240C243B2411244024162445242B2DAB
:106870002F2D6C2D7E2D892D942D972D972D972DB5
:10688000372D372D062E092E0D2E362E632E662E11
:04689000682E952EAB
:10689400E10039000021007F220003490003FFFFCB
:1068A40000FF00390501F4F5680F64127712A30F95
:1068B4007C125C12000000010000000000000005D2
:1068C40001000000050600000000000000000001B7
:1068D4000B000000000000080C0000000000000095
:1068E4000000050904140000000000000118000065
:1068F400000000000119000000000000011A00005F
:1069040000000000091B000000000000012400003A
:10691400000000000C250000000000000000010041
:10692400E413F413321400000001FF00FF78442242
:106934006D3B011901AC009101AA01CA01000810C4
:106944001818100800FF0502000B0C15161F200A6A
:106954000D14171E21090E13181D22080F12191CDD
:10696400230710111A1BFF2F30393A43442E3138B4
:106974003B42452D32373C41462C33363D40472B74
:1069840034353E3FFF60281014300A5012583C380A
:1069940039183C2039003000240018000C100C1069
:1069A400181024103030374039202D202120152094
:1069B4000930073013301F302B503B6040402D40CE
:1069C4002140154009500A50165022502F8028D0DB
:1069D40014B00A9012883CA839C83CC039E030E0B1
:1069E40024E018E00CD00CD018D024D030B037A05C
:1069F40039C02DC021C015C009B007B013B01FB0F5
:106A04002B903B8040A02DA021A015A009900A90B6
:106A1400169022902F0802020202020204040404C7
:106A24000404040404040404040404040404040422
:106A3400040404040404040404080202020202021A
:106A44000404040404040404040404040404040402
:106A5400040404040404040404040404040031319C
:106A6400295A1B750A42415345004C4F5745520061
:106A740052414953450041444A5553540000D502FC
:106A8400010101DA02010202E002010003E602014F
:106A94000300FF0100010000FFFF0000010001FFEF
:106AA4000046076697C63435F6F731333236E200CE
:106AB400E900EA00B500B600B700CD008301CC00C0
:106AC4008A01920194012102230224022502260252
:106AD40027022A02B300B4006F0070009F01CB01AB
:106AE4009F02A002E200E900EA00B500B600B70088
:106AF400CD008301CC008A0192019401210223027A
:106B040024022502260227022A02B300B4006F00E1
:0A6B140070009F01CB019F02A00258
:00000001FF
